:020000040800F2
:10000000181A002001010008090100080B0100086E
:100010000D0100080F010008110100080000000098
:1000200000000000000000000000000013010008B4
:100030001501000800000000170100081901000860
:100040001B0100081B0100081B0100083D2B0008D4
:100050001B0100081B0100081B0100088912000891
:100060001B0100081B0100081B010008610E0008AD
:100070001B0100081B0100081B0100081B010008F0
:100080001B0100081B0100081B0100081B010008E0
:100090001B0100081B0100081B0100081B010008D0
:1000A0001B0100081B0100081B0100081B010008C0
:1000B0001B01000891340008793900081B01000871
:1000C0001B0100081B0100081B0100081B010008A0
:1000D0001B010008913B00081B0100081B010008E0
:1000E0001B0100081B0100081B010008DFF80CD0F1
:1000F00000F080FC0048004789570008181A0020CB
:100100000648804706480047FEE7FEE7FEE7FEE7B1
:10011000FEE7FEE7FEE7FEE7FEE7FEE7D133000875
:10012000ED00000840EA01039B0703D009E008C97D
:10013000121F08C0042AFAD203E011F8013B00F8AC
:10014000013B521EF9D27047F0B480EA0102D40F8D
:100150004200B2EB410F02D20246084611464A0065
:1001600042D0C30DDDB2C1F3C752AD1A202D35DA2E
:10017000C1F3160141F4000204B15242C5F1200658
:1001800002FA06F12A411044B3EBD05F23D0C4B188
:10019000012DA0EBC35009DCF0BC4FF0004202EA95
:1001A000C352DBB200F5000000F069BB400000F173
:1001B000807000EBC350A0F1807040EAD17049001C
:1001C00009E0490841EAC071A0EBC35000F5000006
:1001D000400800EBC350F0BC00F048BB6142012274
:1001E00002EB4101001BF6E7F0BC704781F00041D3
:1001F000AAE780F00040A7E780EA010210B502F00C
:100200000043400022D04A001FD0010E01EB1261D2
:10021000C0F35600C2F3560240F4000042F400025C
:10022000A0FB022000047F39140400D0401C50EAD7
:10023000124001D44000491EC2B20C0604EBD0109B
:10024000401C4008802A02D003E0002010BD20F0AE
:100250000100002900DA0020184310BD30B480EA04
:10026000010202F0004530F0004221F0004013D0BE
:1002700090B1C30DD40DC2F31601C0F31600E41AF9
:1002800041F4000140F400027D34914201D3641C2A
:1002900000E04900002C02DA30BC002070474FF427
:1002A00000000023914201D3891A034340084FEA1A
:1002B0004101F7D151B1914202D14FF0004105E027
:1002C00002D24FF0010101E06FF0010103EBC450D5
:1002D000284430BC00F0CABA2DE9FE4F804681EABE
:1002E0000300C00F0C46009021F0004123F00045B0
:1002F000B8EB0200A94105D24046214690461C4673
:100300000B46024623F00040104347D0270DC7F3A9
:100310000A00C3F30A510290401A019040286BDA98
:10032000C3F3130040F4801B0098924620B10023D1
:10033000D2EB030A63EB0B0B01985946C0F1400264
:10034000504600F062FA06460D4650465946019A5C
:1003500000F07AFA10EB08006141002487EA11529C
:1003600084EAE7731A4340D0009A62B3019A012AE3
:100370004FEA075215DC001B61EB02014FF000420F
:1003800002EA0752CDE90042001C41F580113246D5
:100390002B4600F0B1FA03B0BDE8F08F404621468D
:1003A000F9E7001B61EB0201001C41F58013001806
:1003B0005B412018A2F5001747EB030140EAD57016
:1003C000B6196D4111E06D084FEA360645EAC07571
:1003D0004FEA0752001B61EB0201001C41F580113E
:1003E00049084FEA30000019514132462B4603B00C
:1003F000BDE8F04F00F071BA0098012240000023E0
:10040000D0EB020263EBE073009821464FEAE07400
:10041000B8EB000061EB0401E9E783F000435BE720
:1004200081F0004158E72DE9FE4F81EA030404F012
:10043000004421F0004100944FF0000B23F00043F2
:1004400050EA01045ED052EA03045BD0C3F30A54BD
:10045000C1F30A552C44A4F2F3340194A0FB0254D6
:10046000C1F3130141F48011C3F3130343F4801368
:1004700001FB024400FB034E840A970A44EA8154BC
:1004800047EA8357A4FB076802958D0A05FB078599
:100490004FEA932C04FB0C542705029D4FEA0658A3
:1004A00047EA1637B5EB08056EEB070C870E920E80
:1004B00047EA811742EA8312A7FB0201B6EB0B0160
:1004C00064EB00042B0D43EA0C335E1844EB1C5024
:1004D000DA465146E7FB0201C5F313044FEA0B333A
:1004E00043EA14534FEA0432019C43EA0603A4F1A1
:1004F0000C040294009CCDE900B400F0FDF903B0B7
:10050000BDE8F08F00200146F9E72DE9F04D81EAC2
:10051000030404F0004B21F0004514464FF0000A9C
:1005200023F0004150EA050220D054EA01021DD018
:10053000C5F30A570246C5F31303C1F31300C1F311
:100540000A5640F4801543F48013A7EB0608101BED
:10055000D64608F2FD3873EB050002D308F1010816
:1005600001E092185B41B8F1000F03DA0020014668
:10057000BDE8F08D00204FF48011064684460EE061
:10058000171B73EB050705D3121B63EB050306432B
:100590004CEA010C49084FEA300092185B4150EADE
:1005A0000107EDD152EA030012D082EA040083EA87
:1005B0000501084305D0101BAB4106D201220023E0
:1005C00006E000224FF0004302E06FF001025310FA
:1005D0001AEB06004CEB085110EB0A0041EB0B0143
:1005E000BDE8F04D00F079B9C10F80EAE070084431
:1005F000CA079623002100F042B996230022114633
:1006000000F03DB90EB5C10F80EAE0700844CA079A
:10061000002140F233438DE80E000A460B4600F0FD
:100620006BF903B000BD0EB540F2334102910021D9
:10063000CDE900110A460B4600F05EF903B000BD9B
:1006400000F0004220F00040C10DC0F3160040F45D
:1006500000007F2901DA00207047962903DCC1F1F0
:100660009601C84001E096398840002AF4D0404203
:10067000704720F00040C10DC0F3160040F40000A8
:100680007F2901DA00207047962903DCC1F1960129
:10069000C840704796398840704770B5C1F30A5218
:1006A00001F000450024C1F3130140F2FF3341F48F
:1006B00080119A4201DA002070BD40F233439A4221
:1006C000A2F2334203DC524200F0AEF800E0904068
:1006D0002C43F1D0404270BDC1F30A5210B5C1F3B2
:1006E000130140F2FF3341F480119A4201DA0020F5
:1006F00010BD40F233439A42A2F2334203DC52422D
:1007000000F092F810BD904010BD00F0004230F0B3
:1007100000400AD0C10D01F56071C0F3160042EA35
:100720000151C2084007114370470020014670473D
:1007300001F0004330B421F0004150EA010206D03C
:100740000A0DA2F56072C1F31301002A02DC30BC6D
:1007500000207047440F44EAC104C100E01830BCD7
:1007600000EBC25000F082B8002801DBC0F100406D
:10077000002901DBC1F100418142704730B50B46D1
:10078000014600202022012409E021FA02F59D42C1
:1007900005D303FA02F5491B04FA02F52844151E95
:1007A000A2F10102F1DC30BD2DE9F05F0546002029
:1007B00092469B4688460646814640241BE02846D2
:1007C00041464746224600F02FF853465A46C01A83
:1007D000914110D311461846224600F016F82D1A02
:1007E00067EB01084F4622460120002100F00DF87A
:1007F00017EB00094E41201EA4F10104DFDC48463E
:1008000031462A464346BDE8F09F202A04DB203AC1
:1008100000FA02F1002070479140C2F1200320FA53
:1008200003F3194390407047202A04DB203A21FA51
:1008300002F00021704721FA02F3D040C2F12002F9
:100840009140084319467047202A06DBCB17203A0F
:1008500041FA02F043EAE07306E041FA02F3D040C5
:10086000C2F1200291400843194670470029A8BFF1
:100870007047401C490008BF20F00100704710B4C9
:10088000B0FA80FC00FA0CF050EA010404BF10BC7E
:10089000704749B1CCF1200421FA04F411FA0CF1AB
:1008A00018BF012121430843A3EB0C01CB1D4FEAE4
:1008B00000614FEA102042BF002010BC704700EBDF
:1008C000C35010440029A4BF10BC7047401C49000D
:1008D00008BF20F0010010BC704710B5141E73F162
:1008E000000408DA401C41F1000192185B411A43F0
:1008F00001D120F0010010BD2DE9F04D92469B463C
:1009000011B1B1FA81F202E0B0FA80F220329046E1
:10091000FFF77BFF04460F4640EA0A0041EA0B015D
:1009200053465A46084313D0114653EA010019D0E2
:10093000C8F140025046FFF777FF05460E46504685
:1009400059464246FFF761FF084305D0012004E005
:1009500020463946BDE8F08D0020054346EAE076A2
:100960002C4337430A986305E40AA0EB08000022F1
:10097000FD0A44EA47540A3002D500200146E9E75F
:10098000010510196941DDE9084500196941BDE813
:10099000F04DA2E7C1F30A52C1F3130140F2FF3355
:1009A00041F480119A4202DA00200146704740F279
:1009B00033439A42A2F2334202DC5242FFF734BF81
:1009C000FFF723BF30B5041E71F1000404DB4FF0C4
:1009D0000044404264EB0101141E73F1000405DB86
:1009E0001C464FF00043524263EB0403994208BF98
:1009F000904230BD064C074D06E0E06840F0010330
:100A000094E8070098471034AC42F6D3FFF772FB26
:100A1000E8B3000808B4000870B58C1810F8015B42
:100A200015F0070301D110F8013B2A1106D110F887
:100A3000012B03E010F8016B01F8016B5B1EF9D18B
:100A40002B0705D40023521E0DD401F8013BFAE711
:100A500010F8013BCB1A921C03E013F8015B01F87C
:100A6000015B521EF9D5A142D8D3002070BD21B13F
:100A7000826842F00102826003E0826822F0010293
:100A80008260704721B1826842F48072826003E024
:100A9000826822F480728260704721B1826842F4D9
:100AA0008012826003E0826822F4801282607047C4
:100AB000014600208A6802F004020AB1012000E029
:100AC00000207047014600208A6802F008020AB13F
:100AD000012000E00020704730B5024600200023CE
:100AE00050680F4C20400D790C6844EA05242043DF
:100AF000506090680B4C2040D1E902542C434D7952
:100B000044EA450420439060D06A20F470000C7CD5
:100B1000641EE4B2234340EA0350D06230BD0000BB
:100B2000FFFEF0FFFDF7F1FF00B585B000F0B8FC67
:100B30000121480201F036FE0020009001208DF8CE
:100B400004008DF805004FF4C020029000200390AF
:100B500009208DF8100069462E48FFF7BDFF4FF4BD
:100B6000004001F0E3FD072301220021294800F0A5
:100B700053F8072302220121264800F04DF80723ED
:100B800003220221234800F047F80723042203210F
:100B9000204800F041F80723052204211D4800F0F9
:100BA0003BF80723062205211A4800F035F80723F1
:100BB0001A460621174800F02FF807230822194685
:100BC000144800F029F8072309220821114800F0F1
:100BD00023F801210F48FFF755FF01210D48FFF7CA
:100BE00046FF0C4800F074F800BF0A48FFF76AFFA0
:100BF0000028FAD1074800F070F800BF0548FFF759
:100C000057FF0028FAD101210248FFF746FF05B03F
:100C100000BD000000240140F0B504460D46002050
:100C20000021092D11DDE068A5F10A0606EB460753
:100C3000072606FA07F18843A5F10A0606EB4606E1
:100C400003FA06F10843E0600CE0206905EB450774
:100C5000072606FA07F1884305EB450603FA06F175
:100C600008432061072A0FDA606B561E06EB8607E1
:100C70001F2606FA07F18843561E06EB860605FA7C
:100C800006F10843606322E00D2A0FDA206BD61FBD
:100C900006EB86071F2606FA07F18843D61F06EBE8
:100CA000860605FA06F10843206310E0E06AA2F127
:100CB0000D0606EB86071F2606FA07F18843A2F108
:100CC0000D0606EB860605FA06F10843E062F0BD64
:100CD000816841F0080181607047816841F004013A
:100CE0008160704708B50121042001F05BFD4FF4DD
:100CF0008060ADF8000010208DF8030003208DF80F
:100D000002006946044800F009FC4FF48061024883
:100D100000F0E1FC08BD00000008014010B5012012
:100D200001F060FD002001F05DFD10BD08B5014639
:100D3000002000900348009000980844009000981C
:100D4000008808BD006C004008B500220092044AEB
:100D50000092009A02440092009A116008BD0000BF
:100D6000006C004070B588B0054600246FE0C4EB0D
:100D7000C400394901EB800005EB0413D3E901629B
:100D80001968DB68C0E90162C3600160C4EBC4019B
:100D9000314A02EB8101C868012101F003FDC4EB77
:100DA000C4002D4901EB8000008901A921F824002D
:100DB000C4EBC400284911F8200001A901EB84010B
:100DC000C87001AA02EB8401C4EBC402224B03EBFE
:100DD0008202506800F0A2FB0120C4EBC4011E4A4D
:100DE00002EB810108740021C4EBC40002EB800017
:100DF0004174C4EBC40002EB80008174C4EBC400F6
:100E0000114611F82000482806D10021C4EBC40087
:100E100002EB8000C17406E00121C4EBC4000E4A5D
:100E200002EB8000C1740021C4EBC4000A4A02EB4B
:100E300080000175C4EBC40002EB800041750749D6
:100E4000C4EBC40002EB80008161601CC4B2072CBB
:100E50008DDB08B070BD0000CC100020ED1800083C
:100E60002DE9F04F89B04FF0000B022000F0CEF9D1
:100E700000287CD0DA4617E0584890F85F0038B177
:100E80005146574800F02BFC564921F81A0007E05C
:100E9000CAF10301524800F022FC524921F81A001D
:100EA0000AF101001FFA80FABAF1040FE4DB4FF0F7
:100EB000040A0AE051464A4800F011FC494921F869
:100EC0001A000AF101001FFA80FABAF1080FF1DBEB
:100ED0004FF0000A36E04148523010F80A003F4C0B
:100EE000223404EB4A04009023883C4C123404EB77
:100EF0004A042288394CA41C04EB4A042188394C4A
:100F000034F81A0004F0B8FC3449323101EB8A019C
:100F100009680844344921F81A00084630F81A00D4
:100F2000A0F5FA70012101EB4A01304A22F81100C4
:100F30002D4830F81A0058441FFA80FB0AF10100CE
:100F40001FFA80FABAF1080FC5DB44F62060A0EB67
:100F50000B002649488407F03DF82049B1F86000AD
:100F6000FFF761FBCDE9040108211D4800E032E0F4
:100F700000F0B5FB0190FFF745FB06464FF06632E7
:100F80001B4BFFF750FA044600221A4BFFF74BFAAF
:100F9000CDE90201DDE90423FFF745FA0022164BF3
:100FA000CDE90601FFF7B1FA8046FFF7C1FB13490F
:100FB00008600A48D0F85B1010480068FFF7D4FBBF
:100FC00003D201200E49087002E000200C4908708D
:100FD000022000F05BF809B0BDE8F08FA4150020F6
:100FE000F80B0020AC0C0020BC0C0020E00A002014
:100FF00066660A40000008400C3E4F411400002085
:101000001800002000B58DB00121084601F09AFBC0
:101010001B4800F055F81B4802901B480390002025
:1010200004905A20059000200690802007904000F0
:1010300008908000099020200A9000020B90002068
:101040000C9002A90E4800F000F9012202210C4880
:1010500000F0F2F80B208DF8040001208DF8050057
:1010600000208DF8060001208DF8070001A800F08F
:10107000C3FD0121024800F017F80DB000BD0000CB
:10108000080002404C240140F80B002000F0805181
:1010900011B10349086001E002494860704700004F
:1010A000040402400000024021B1026842F0010243
:1010B000026004E002684FF6FE731A400260704757
:1010C00001684FF6FE72114001600021016041602D
:1010D0008160C1604B49884208D14A490839496852
:1010E00041F00F01474A083A51608AE045491431FE
:1010F000884208D143490839496841F0F001414A22
:10110000083A51607DE03F492831884208D13D4985
:101110000839496841F470613A4A083A516070E010
:1011200038493C31884208D136490839496841F488
:101130007041344A083A516063E032495031884284
:1011400008D130490839496841F470212D4A083ADC
:10115000516056E02B496431884208D12949083949
:10116000496841F47001274A083A516049E025492D
:101170007831884208D123490839496841F07061C3
:10118000204A083A51603CE01F49884206D1011FBD
:10119000096841F00F01021F116032E01A49143151
:1011A000884208D11849091F096841F0F001164A20
:1011B000121F116025E014492831884208D11249D4
:1011C000091F096841F470610F4A121F116018E08D
:1011D0000D493C31884208D10B49091F096841F487
:1011E0007041094A121F11600BE0074950318842D3
:1011F00007D10549091F096841F47021024A121FED
:1012000011607047080002400804024001460020B7
:10121000002201F0805313B1054B1A6801E0054B21
:101220001A6802EA01030BB1012000E000207047B8
:1012300000040240000002401AB103680B4303603F
:1012400002E003688B430360704710B50022026818
:1012500047F6F0739A430C6A8B6823430C69234367
:101260004C6923438C692343CC6923434C6A234351
:101270008C6A23431A430260CB6843600B68836027
:101280004B68C36010BD000010B5012003F000FBE7
:10129000012012490880124800681249D1F828112B
:1012A00088420BD110480078012803D10B200B494C
:1012B00048800EE00620094948800AE00A48007884
:1012C000012803D10C200549488002E0072003498A
:1012D0004880022000F00AF810BD00001A0000202B
:1012E000048121420080214223000020014908603E
:1012F0007047000014040140002123498279002A2C
:101300003AD00A46126803689A430B461A600A1DCF
:10131000126803689A430B1D1A60027911440A6827
:1013200003681A430A60184A0832126803689A432D
:10133000154B08331A601A1D126803689A43124B42
:101340000C331A604279102A0ED11A1F12680368F2
:101350001A430D4B08331A601A1D126803681A43AA
:10136000094B0C331A600DE00749427911440A68B1
:1013700003681A430A6005E0027911440A680368A9
:101380009A430A60704700000004014030B50446EB
:1013900004254FF4302000F06FF80546042D17D1D6
:1013A0000C48006940F002000A490861084644619F
:1013B000006940F0400008614FF4302000F05CF814
:1013C00005460448006941F6FD710840014908617D
:1013D000284630BD0020024004200B49C96801F0B6
:1013E000010109B101200EE00749C96801F00401BB
:1013F00009B1022007E00449C96801F0100109B1F0
:10140000032000E0042070470020024003480069E8
:1014100040F0800001490861704700000020024050
:1014200070B504460D460426F00200F025F8064685
:10143000042E11D10948006940F0010007490861F4
:101440002580F00200F018F806460448006941F6CD
:10145000FE71084001490861304670BD002002401D
:1014600002480349486003484860704723016745C4
:1014700000200240AB89EFCD00B502460423FFF700
:10148000ABFF034603E0FFF7A7FF0346521E012B05
:1014900001D1002AF7D102B90523184600BD00008A
:1014A00008B501210C2001F07DF9FF20ADF8000006
:1014B00003208DF8020000208DF8030069460548DE
:1014C00000F02CF80120ADF800006946024800F059
:1014D00025F808BD00080140000C014030B500228D
:1014E0008B071C0F0F2303FA04F20B4B8C1053F8DD
:1014F00024309343084C8D1044F8253023468C103B
:1015000053F824308C07240F00FA04F42343024CD0
:101510008D1044F8253030BD080001402DE9F04120
:10152000024600250026002000230024002791F811
:1015300003C00CF00F0591F803C00CF0100CBCF1C7
:10154000000F03D091F802C04CEA050591F800C0E5
:10155000BCF1000F31D0146800202BE04FF0010CDB
:101560000CFA00F3B1F800C00CEA03069E4220D149
:1015700083004FF00F0C0CFA03F7BC4305FA03FC91
:101580004CEA040491F803C0BCF1280F06D14FF0D7
:10159000010C0CFA00FCC2F814C00AE091F803C078
:1015A000BCF1480F05D14FF0010C0CFA00FCC2F859
:1015B00010C0401C0828D1D31460B1F800C0BCF1A1
:1015C000FF0F34DD546800202EE000F1080C4FF0CE
:1015D000010808FA0CF3B1F800C00CEA03069E42B9
:1015E00021D183004FF00F0C0CFA03F7BC4305FA2E
:1015F00003FC4CEA040491F803C0BCF1280F05D1A8
:1016000000F1080C08FA0CF8C2F8148091F803C035
:10161000BCF1480F07D100F1080C4FF0010808FA9F
:101620000CF8C2F81080401C0828CED35460BDE8E6
:10163000F0810000F0B50A460023002400210025B7
:1016400000F00046B6F1004F02D11D4EF16901E0F5
:101650001B4E7168C0F3034583B200F44016B6F523
:10166000401F08D121F07061154E766826F0706633
:10167000134F7E6012E000F48016B6F5801F06D18D
:10168000032606FA05F4A14341F0706106E0460D19
:10169000360103FA06F6B14341F0706122B1460DFE
:1016A000360103FA06F6314300F00046B6F1004F6A
:1016B00002D1034EF16101E0014E7160F0BD000006
:1016C000000001400246002093680B400BB101204E
:1016D00000E0002070474161704701617047F0B53C
:1016E00085B003460C46002107E0092505FB0145AE
:1016F00033F815502DF81150491C0A29F5DB00224A
:1017000018E0002111E03DF811604D1C3DF8155026
:10171000AE4209DD3DF811004D1C3DF815502DF885
:1017200011504D1C2DF81500491CC2F109058D42C0
:10173000E9DC521C092AE4DBBDF80A60BDF80C7034
:10174000F51905EBD576701005B0F0BD70B5002425
:101750002DE0C4EBC400174901EB8000007C00B908
:1017600023E0C4EBC400134901EB8005C4EBC400C3
:1017700001EB8000866995E80F00B047C4EBC40117
:101780000C4A02EB8101C97C884206D10121C4EBDD
:10179000C40002EB8000817406E00021C4EBC400A9
:1017A000044A02EB8000817400BF601CC4B2072CA5
:1017B000CFDB70BDCC10002010B54FF4807109480C
:1017C000FFF78BFF4FF400710648FFF786FF4FF4D9
:1017D00000710448FFF77FFF4FF480710148FFF765
:1017E0007AFF10BD000C014010B54FF4807107481E
:1017F000FFF773FF4FF400710448FFF76CFF4FF4DD
:1018000000710248FFF769FF10BD0000000C0140A5
:1018100010B54FF480710448FFF75FFF4FF48071FB
:101820000148FFF758FF10BD000C014002464FF081
:10183000FF3300210EE00C4830F81100904201D136
:101840000B4609E0084830F81100904200DD03E043
:10185000481C81B22B29EEDB00BF002B01DA0020EF
:1018600070470120FCE700007C0600200146CA17F3
:1018700001EB92729210A1EB820292B9642091FB6B
:10188000F0F200FB121050B94FF4C87091FBF0F267
:1018900000FB121008B9012070470020FCE701206E
:1018A000FAE70020F8E7000000B59DB003F082F8E9
:1018B00070220B4901A8FEF735FC01A8FFF752FA88
:1018C0000121084600F06EFF01210648FFF7B2FE35
:1018D0000548406820F02000034948601DB000BD65
:1018E000F48C000800023000002004E01FB5BDF8B1
:1018F00008100198FFF7E6FE04B010BD1CB511A159
:1019000003C9CDE90001082001F0F2FB0522694678
:10191000302000F02BF905226946102000F090F8E5
:10192000002406E01DF80400A52800D003E0601C98
:10193000C4B2052CF6DB00BF052C01D001201CBD74
:101940000020FCE7A5A5A5A5A500000000B587B06F
:1019500001211C2000F026FF4FF48050ADF8180044
:1019600010208DF81B0003208DF81A0006A92948C5
:10197000FFF7D4FD4FF48070ADF8180006A9264893
:10198000FFF7CCFD4FF40070ADF8180028208DF85B
:101990001B0006A92048FFF7C1FD4FF440711E4807
:1019A000FFF799FE4FF480511A48FFF794FE01F0BB
:1019B0002BFB0021194801F0AFFB0020ADF804001B
:1019C0004FF48270ADF806000020ADF80800ADF8C5
:1019D0000A00ADF80C004FF40070ADF80E001820AE
:1019E000ADF810000020ADF812000720ADF814008B
:1019F00001A90A4801F0AAFB0121084801F08CFB6B
:101A000000200749086001200649C1F8B00107B06D
:101A100000BD0000000C01400008014000380040FB
:101A2000A00121420080214210B500200349086036
:101A30000C21202000F0B8F810BD0000A0012142C8
:101A40002DE9F04107460D46164600200A49086078
:101A5000384601F023FB8046002405E0FF2001F01A
:101A60001DFB2855601CC4B2B442F7DB01200249BB
:101A700008604046BDE8F081B081214270B504465F
:101A8000002007490860204601F008FBFF2001F014
:101A900005FB054601200349C1F8B001284670BD89
:101AA000B08121420080214210B504460020144933
:101AB000086005221349302000F058F80522124929
:101AC0002A2000F053F80121212000F06DF80121B7
:101AD000222000F069F81A21242000F065F828215E
:101AE000252000F061F82146262000F05DF80E2147
:101AF000202000F059F801200449C1F8A00110BDD0
:101B0000A0012142648D0008698D00080000214277
:101B100070B50546102001F0EBFA0020114908606D
:101B200020222946A02000F021F801200E49C1F80A
:101B3000A0010720FFF7A2FF04462146272000F05E
:101B400033F804F0100028B1FF21E12000F02CF858
:101B5000102070BD04F0200008B12020F9E7FF201C
:101B6000F7E70000A0012142000021422DE9F041E9
:101B700007460C46154600200A490860384601F021
:101B80008DFA8046002605E014F8010B01F086FA74
:101B9000701CC6B2AE42F7DB012002490860404625
:101BA000BDE8F081B081214270B505460C460020A9
:101BB00007490860284601F071FA0646204601F000
:101BC0006DFA01200349C1F8B001304670BD000034
:101BD000B08121420080214208B51E208DF800000E
:101BE00000208DF801008DF8020001208DF803001F
:101BF000684600F001F808BD70B5002100230F22EF
:101C0000C47804B3154C246804F4E064C4F5E064BB
:101C1000210AC1F10403CA40447804FA03F184782C
:101C20001440214309010E4C0678A155047804F0B4
:101C30001F050124AC4005786D11AD0005F1E025CC
:101C4000C5F8004109E0047804F01F050124AC4008
:101C5000044D0678761145F8264070BD0CED00E085
:101C600000E400E080E100E002490143024A116023
:101C7000704700000000FA050CED00E070B500248C
:101C800018E004F1B000002100F001FB002108463B
:101C900000F0FDFA0021102000F0F9FA002505E01F
:101CA0000121002000F0F3FA681CC5B2802DF7DB9B
:101CB000601CC4B2082CE4DB70BD000000200CE006
:101CC000002106E00022064B03EBC0035A544A1CD5
:101CD000D1B20829F6DB421CD0B28028F0DB704775
:101CE00099110020F0B5144600267F2801DC3F2919
:101CF00000DDF0BD0B46CF1701EB5777FF10C7F1A2
:101D00000707FAB2CF1701EB5777FF10A1EBC70710
:101D1000FDB2C5F107070123BB40DEB24CB10A4B4F
:101D200003EBC0039B5C3343074F07EBC007BB5477
:101D300008E0054B03EBC0039B5CB343024F07EB8A
:101D4000C007BB5400BFD4E7991100202DE9F04F24
:101D500006460C4617469846A346002530E017F87D
:101D600005904FF0000A25E009F0800028B12146D7
:101D700030460A9AFFF7B6FF09E00A9808B9012031
:101D800000E00020024621463046FFF7ABFF4FF649
:101D9000FF7000EA4909601CC4B2A4EB0B0109986A
:101DA000814203D15C46701CC6B206E00AF1010014
:101DB0001FFA80FABAF1080FD6DB00BF681C85B2A3
:101DC000099908FB01F0C11700EB5171B5EBE10F68
:101DD000C5DBBDE8F08F2DE9F04706460F4690467B
:101DE0009946DDF820A034460CE03D4606E0524618
:101DF00029462046FFF776FF681CC5B24D45F6DD43
:101E0000601CC4B24445F0DDBDE8F08708B501218F
:101E1000092000F0C7FC01210220FFF70BFC4FF462
:101E20004070ADF8000010208DF8030003208DF8FD
:101E3000020069463B48FFF771FB4FF44071394897
:101E4000FFF74BFC0A2002F023FD0021AE2000F03A
:101E50001EFA0021084600F01AFA0021102000F0B6
:101E600016FA0021402000F012FA0021B02000F004
:101E70000EFA0021812000F00AFA0021FF2000F074
:101E800006FA0021A12000F002FA0021A62000F0AD
:101E9000FEF90021A82000F0FAF900213F2000F00F
:101EA000F6F90021C02000F0F2F90021D32000F063
:101EB000EEF90021084600F0EAF90021D52000F0F3
:101EC000E6F90021802000F0E2F90021D82000F09E
:101ED000DEF90021052000F0DAF90021D92000F018
:101EE000D6F90021F12000F0D2F90021DA2000F02B
:101EF000CEF90021122000F0CAF90021DB2000F009
:101F0000C6F90021302000F0C2F900218D2000F038
:101F1000BEF90021142000F0BAF90021AF2000F032
:101F2000B6F908BD000C014070B500241BE004F1B7
:101F3000B000002100F0ABF90021084600F0A7F93D
:101F40000021102000F0A3F9002508E0074901EB6B
:101F5000C501085D012100F09AF9681CC5B2802D09
:101F6000F4DB601CC4B2082CE1DB70BD99110020C9
:101F70002DE9F84F80460F4616461C46BA462046C5
:101F8000E31704EB5373DB1021464FEAE47C04EBC8
:101F90005C7C4FEAEC0CA4EBCC0CBCF1000F02D043
:101FA0004FF0010C01E04FF0000C6344224604EBBB
:101FB000D27C4FEA6C0C03FB0CF303F0FF0BA6F191
:101FC0002000C6B200254EE00C2C07D106EB4600DF
:101FD000274901EB8000405D009013E0102C05D1F3
:101FE000244800EB0610405D00900BE0182C07D150
:101FF00006EBC600204901EB8000405D009001E047
:10200000BDE8F88F4FF0000927E0009800F080004D
:1020100028B1394640460A9AFFF764FE09E00A985B
:1020200008B9012000E00020024639464046FFF78B
:1020300059FE00984006000E0090781CC7B2A7EB2E
:102040000A00A04205D1574608F1010000F0FF0840
:1020500006E009F1010000F0FF09B9F1080FD4DB37
:1020600000BF681CC5B25D45AEDB00BFC8E700001D
:102070006E8D0008E2910008D29700082DE9FE4F0E
:1020800006460D4617461C46DDF830A00195204651
:10209000E21704EB5272D2102146E31704EB53739C
:1020A000DB10A4EBC3030BB1012300E000231A44AF
:1020B0006243D2B200920C2C05D107EB47002549B0
:1020C00001EBC0090AE0102C03D1234800EB4719AB
:1020D00004E007EBC700214901EBC0094FF00008FD
:1020E00032E019F808B00020029025E00BF08000E3
:1020F00028B1E9B2F0B25246FFF7F4FD0AE0BAF1B6
:10210000000F01D1012300E000231A46E9B2F0B22A
:10211000FFF7E8FD4FEA4B604FEA106B681C85B291
:102120000198281AA04203D1019D701C86B206E0D6
:102130000298401CC0B2029002980828D6DB00BF6B
:1021400008F1010000F0FF0800988045C9DBBDE8F8
:10215000FE8F00002EA5000846A5000886B30008E3
:102160002DE9F8430546884616461F46DDF82090BF
:1021700000240BE0CDF80090325D05EB041188B22D
:1021800010234146FFF77AFF601CC4B2BC42F1DB6A
:10219000BDE8F8832DE9FF4F82B0074691461E4601
:1021A000DDE90F5A00200190002438E0301B401E6A
:1021B000C1B20A2005F076FDB9FBF0F00A21B0FBB0
:1021C000F1F201FB12080198B0B9701EA04213DDB4
:1021D000B8F1000F0ED1AB4605EBDB71491001FBE6
:1021E0000471C8B22B462022CDF800A00399FFF756
:1021F000BFFE12E001200190AB4605EBDB714910F8
:1022000001FB0471C8B208F13001CAB22B46CDF807
:1022100000A00399FFF7ACFE00BF601CC4B2B4423B
:10222000C4DB06B0BDE8F08F2DE9F84306460F4643
:1022300015461C46DDF8208021E004EBD4714910DE
:10224000C1F18001B14202DA00263819C7B2C4F1E7
:102250004000B84204DA002006460746FFF70EFDAC
:10226000CDF800802A78234639463046FFF780FEB5
:10227000204604EBD07106EB6101CEB26D1C2878CC
:102280007E2802DC28782028D7DABDE8F88370B5EC
:1022900004460D461DB1E0B201F01EFE02E0E0B2C0
:1022A00001F004FE70BD000010B5F1484088801FA9
:1022B000072856D2DFE800F00F041A3745545300C0
:1022C000EC48007800EB4000EB4901EB80004078DF
:1022D000E849087045E0E748007800EB4000E6492F
:1022E00001EB80008078E34908703AE0E148047827
:1022F000007800EB4000E04901EB8000C078DD4948
:1023000008702046FFF792FA60B1DA480078FFF7CC
:102310008DFA38B1D948007808B9012000E00020D2
:10232000D64908701DE0D348007800EB4000D24940
:1023300001EB80000079CF4908700020CF49087078
:102340000FE0CC48007800EB4000CB4901EB800067
:102350004079C84908700020C849087001E000E0D1
:1023600000BF00BFC348007880B9C548007868B195
:10237000C3480078412804D0C1480078C14908808A
:1023800002E03220BF490880FFF798FCB948007886
:1023900040B1BB48007828B9BA480078B549087000
:1023A000FFF78CFCB3480078012819DBB1480078AE
:1023B000092815DCB2480078012801DA012000E084
:1023C0000020AF490978092901DD012100E0002141
:1023D000084328B144236A220921082003F0DAF9CE
:1023E000A44800780A2815DBA2480078112811DCDF
:1023F000A34800780A2801DA012000E00020A04963
:102400000978112901DD012100E00021084308B10C
:1024100004F04AF897480078122815DB95480078B0
:10242000192811DC96480078122801DA012000E012
:10243000002093490978192901DD012100E00021DC
:10244000084308B104F048F88A4800781A2815DBD8
:10245000884800781D2811DC894800781A2801DA9C
:10246000012000E00020864909781D2901DD0121B5
:1024700000E00021084308B1FFF720FC7D48007808
:102480001E2815DB7B480078212811DC7C48007869
:102490001E2801DA012000E000207949097821296D
:1024A00001DD012100E00021084308B1FFF706FC2F
:1024B00070480078222815DB6E480078242811DC4B
:1024C0006F480078222801DA012000E000206C49E2
:1024D0000978242901DD012100E00021084308B129
:1024E000FFF7ECFB63480078252815DB614800788E
:1024F0002C2811DC62480078252801DA012000E050
:1025000000205F4909782C2901DD012100E000212C
:10251000084308B103F0D4FF564800782D2805D1B0
:10252000574800782D2801D0FFF7C8FB51480078A4
:102530002E2819DB4F480078332815DC50480078E6
:102540002E2801DA012000E000204D4909783329C6
:1025500001DD012100E00021084328B10923082200
:102560003521342003F016F942480078342815DB71
:1025700040480078362811DC41480078342801DAD8
:10258000012000E000203E490978362901DD0121C3
:1025900000E00021084308B1FFF790FB35480078C0
:1025A000372815DB33480078392811DC34480078A7
:1025B000372801DA012000E0002031490978392963
:1025C00001DD012100E00021084308B1FFF776FB9F
:1025D000284800783A2815DB264800783C2811DC8A
:1025E000274800783A2801DA012000E00020244939
:1025F00009783C2901DD012100E00021084308B1F0
:10260000FFF75CFB1B4800783D2815DB1948007874
:102610003F2811DC1A4800783D2801DA012000E04B
:102620000020174909783F2901DD012100E0002140
:10263000084308B1FFF742FB0E480078412805D156
:102640000F480078412801D0FFF738FB094800788F
:102650000B49097888420AD00649097801EB410103
:10266000054A02EB810188688047FFF75DFC10BDD9
:102670001A0000202600002038030020230000203C
:10268000270000202400002008B50121102000F0C0
:1026900089F84FF40050ADF8000003208DF80200D7
:1026A00010208DF8030069460148FEF737FF08BD8A
:1026B000001001400EB50121042000F053F84FF442
:1026C000FA70ADF804004720ADF800000020ADF826
:1026D0000600ADF8020069460E4801F007FA012233
:1026E00011460C4801F0A7F9FFF7CEFFFFF774FA87
:1026F000094890F86E00012804D10121054801F035
:102700006EF903E00021034801F069F90020034954
:1027100008600EBD00080040A4150020B40122424C
:10272000014908627047000000000E420146002087
:10273000034A506820F4404008435060704700004E
:102740000010024029B1064A52690243044B5A6103
:1027500004E0034A52698243014B5A61704700000A
:102760000010024029B1064AD2690243044BDA61E3
:1027700004E0034AD2698243014BDA6170470000EA
:102780000010024029B1064A12690243044B1A6143
:1027900004E0034A12698243014B1A61704700004A
:1027A0000010024029B1064A92690243044B9A6123
:1027B00004E0034A92698243014B9A61704700002A
:1027C0000010024029B1064AD2680243044BDA6085
:1027D00004E0034AD2688243014BDA60704700008C
:1027E0000010024001490860704700004004424266
:1027F00030B500210022002400232D4D6D6805F026
:102800000C0121B1042905D0082923D105E0294D67
:10281000056022E0274D05601FE0254D6D6805F439
:102820007012234D6D6805F48034022505EB924249
:102830001CB9214D554305600BE01D4D6D6805F435
:1028400000351DB11C4D5543056002E0194D55433F
:10285000056002E0174D056000BF00BF144D6D68B4
:1028600005F0F0010909154D6B5C0568DD40456018
:102870000F4D6D6805F4E061090A104D6B5C456809
:10288000DD4085600A4D6D6805F46051C90A0B4D45
:102890006B5C4568DD40C560054D6D6805F44041E1
:1028A000890B074D6B5CC568B5FBF3F5056130BD61
:1028B0000010024000127A0000093D001C0B0020AD
:1028C0002C0B002010B501460022002300204A11E5
:1028D000012A02D1094C236806E0022A02D1074CE2
:1028E000236A01E0054C636A01F01F020124944051
:1028F0001C400CB1012000E0002010BD001002407F
:1029000000210B4A11700A4A203A82F8201001284F
:1029100002D0042808D103E00121054A117004E027
:102920000521034A117000E000BF00BF704700009E
:102930002010024001490860704700003C044242F8
:102940000249096A0143014A1162704700100240BE
:10295000024909888143014A1180704704280040D8
:102960000348008840F010000149088070470000CB
:1029700004280040034800884FF6EF7108400149E1
:10298000088070470428004070B500260024002508
:1029900000F07CF806463948B6FBF0F43848008869
:1029A000A0423CD036490C8040F2B27510E0284677
:1029B000FEF75CFF40B1B4F5B77F02D3A4F5B7745E
:1029C00004E0681C85B206E0A4F26D14681C85B2B0
:1029D000B4F5B67FEBD800BF2A488580002516E005
:1029E00028498888FEF742FF30B1012D04D11D2C03
:1029F00001D31D3C09E00CE02348405DA04203D810
:102A00002148405D241A00E003E0681C85B21C2CBC
:102A1000E6D200BF681C1B498871601CC87117484A
:102A2000B6FBF0F100FB11641649CC704FF4616005
:102A3000B4FBF0F008704FF46160B4FBF0F100FB00
:102A400011403C21B0FBF1F00E4948704FF4616039
:102A5000B4FBF0F100FB11403C21B0FBF1F201FBB3
:102A60001200084988700B46DA799979988800F045
:102A700029F804490872002070BD0000805101004F
:102A8000D20A00209A150020DAB30008002103487A
:102A90000188001F008841EA004070471C28004060
:102AA00001460020064A12880A40D0B2044A121F8A
:102AB00012880A4012B108B1012000E000207047DE
:102AC00004280040F0B503460C461546642093FBED
:102AD000F0F0C6B2642093FBF0F700FB1730C1B2F0
:102AE000132E02DD01F16400C1B20846CF1701EBDD
:102AF000977701EBA707BAB2072092FBF0F700FB2C
:102B0000172082B25719601EDFF82CC01CF8000095
:102B1000384482B2CF1701EB9777BF10A1EB87073C
:102B20001FB9032C01DA501E82B2072092FBF0F786
:102B300000FB1720C0B2F0BDCEB300080EB50120D7
:102B4000FFF7AEFF08B1FFF71FFF0220FFF7A8FF56
:102B5000A0B10220FFF7FCFEFFF716FF0A488078BD
:102B600009494978084A1278CDE9002102900648BF
:102B7000C3798279818805A001F0C4F90520FFF7A7
:102B8000E7FE00F015F90EBD9A150020416C617248
:102B90006D2054696D653A25642D25642D256420CA
:102BA00025643A25643A25640A00000029B1064AE2
:102BB00012880243044B1A8004E0034A12888243BD
:102BC000014B1A8070470000002800401CB500240B
:102BD00001214FF0C050FFF7C5FD0120FFF7A0FD18
:102BE0000420FEF7A3F845F25001884240D0FEF7DA
:102BF00095F80120FFF784FE04E0601CC4B20A20AF
:102C000001F046FE4120FFF75DFE08B9FA2CF4DB27
:102C1000FA2C01DB01201CBD4FF48070FFF790FE01
:102C20000120FFF787FE00F0C3F800F0CBF8012188
:102C30000846FFF7BBFF00F0BBF8FFF791FE47F631
:102C4000FF7000F0A5F800F0B3F8372032210B2315
:102C50001422CDE90010062140F2E47000F026F8BD
:102C6000FFF788FE45F250010420FEF76DF807E0FB
:102C700000F0A8F801210846FFF798FF00F098F847
:102C800000F004F8FFF780FE0020C4E708B5032039
:102C90008DF8000000208DF801008DF80200012061
:102CA0008DF803006846FEF7A7FF08BD2DE9F05F29
:102CB00006460F4690469946DDE90AAB002440F2ED
:102CC000B270864203DB40F63300864202DD01200B
:102CD000BDE8F09F40F2B2750AE02846FEF7C6FD57
:102CE00010B12048044401E01F480444681C85B228
:102CF000B542F2DB781EC7B2002510E01B48405DEC
:102D000040F2A321484304EBC0143046FEF7AEFD69
:102D100018B1012D01D116480444681C85B2BD428A
:102D2000ECDBA8F1010040F2A321484304EBC014FE
:102D3000C9EB4910C0EB092004EB0014CAEB0A10E0
:102D400004EB80045C4401214FF0C050FFF70AFD02
:102D50000120FFF7E5FC204600F00CF800F028F811
:102D60000020B5E70085E2018033E101DAB3000815
:102D70008051010000B50246FFF7F2FD100C034937
:102D80000880091D0A80FFF7F5FD00BD18280040E6
:102D900000B50246FFF7E4FDC2F303400349088093
:102DA000091D0A80FFF7E6FD00BD0000082800406D
:102DB00000BF0348008800F020000028F9D07047C9
:102DC00004280040074800884FF6F771084005497D
:102DD000088000BF0348008800F008000028F9D0F0
:102DE000704700000428004010B5FEF7AFFC002437
:102DF000E2E0C4EBC400724901EB8000007D30B119
:102E0000012822D0032848D004287CD18EE0C4EBCE
:102E1000C4006B4901EB8000807C01280DD10121A9
:102E2000C4EBC400664A02EB800001750021C4EBCC
:102E3000C40002EB8000417506E00021C4EBC40031
:102E40005F4A02EB80004175B3E0C4EBC4005C490B
:102E500001EB8000807C012812D10321C4EBC40067
:102E6000574A02EB80000175C4EBC40002EB8000FE
:102E700041750021C4EBC40002EB800041740BE0FB
:102E80000021C4EBC4004E4A02EB80000175C4EB84
:102E9000C40002EB800041758BE0C4EBC4004849DC
:102EA00001EB8000807C01280DD00021C4EBC40020
:102EB000434A02EB800001750221C4EBC40002EB1F
:102EC0008000417531E0C4EBC4003D4901EB800056
:102ED000807C012822D1C4EBC40001EB8000407C3F
:102EE000401CC1B2C4EBC400354A02EB80004174FF
:102EF0001E2913DB0421C4EBC40002EB8000017522
:102F0000C4EBC40000E053E002EB800041750021F7
:102F1000C4EBC40002EB8000417406E00021C4EB66
:102F2000C400274A02EB8000417542E0C4EBC400B4
:102F3000234901EB8000807C01280DD00021C4EBE7
:102F4000C4001F4A02EB800001750221C4EBC400DB
:102F500002EB800041752AE0C4EBC400184901EB84
:102F60008000807C01281BD1C4EBC40001EB8000F1
:102F7000407C401CC1B2C4EBC400114A02EB80008B
:102F800041741E290CDB0421C4EBC40002EB800059
:102F900041750021C4EBC40002EB8000417406E0DF
:102FA0000021C4EBC400064A02EB8000417500E03A
:102FB00000BF00BF601CC4B2072CFFF61AAF10BDE3
:102FC000CC10002010B50D48006882B20C490D48A5
:102FD00000F0DAF80A48008841F2111188420BD05B
:102FE00008460749088004F069FE0448006882B278
:102FF0000349044800F0DCF810BD0000DC0A0020A2
:10300000A415002004FC000800B587B001210820A9
:10301000FFF7C8FB01218803FFF7A4FB4FF46040D2
:10302000ADF8180018208DF81B0003208DF81A0049
:1030300006A91848FEF772FA4FF460411548FEF7EA
:103040004CFB0020ADF804004FF48270ADF8060090
:103050000020ADF808000220ADF80A000120ADF80C
:103060000C004002ADF80E003820ADF81000002032
:10307000ADF812000720ADF8140001A9064800F0D1
:1030800065F80121044800F047F8FF2000F006F839
:1030900007B000BD000C01400038004070B5054687
:1030A000002405E0601CC4B2C82C01DD002070BD06
:1030B00002210E4800F03CF80028F3D029460B48C6
:1030C00000F042F8002405E0601CC4B2C82C01DD09
:1030D0000020ECE70121054800F02AF80028F3D091
:1030E000024800F02EF8C0B2E1E7000000380040CE
:1030F00010B50446074800884FF6C77108400549D7
:10310000088008460088204308800121014800F01B
:1031100003F810BD0038004021B1028842F040029F
:10312000028004E002884FF6BF731A4002807047A5
:103130000246002013890B400BB1012000E0002063
:1031400070470146888970478181704710B5002219
:10315000028802F441520B884C8823438C88234315
:10316000CC8823430C8923434C8923438C892343F4
:10317000CC8923431A430280838B4FF2FF74234090
:1031800083830B8A038210BD30B503460C46154677
:10319000002207E0184600F008F824F812009B1CF3
:1031A000501C82B2AA42F5DB30BD01460888704748
:1031B0002DE9F05F80468A461746B8F1006F02D3CA
:1031C0003348804501D3BDE8F09FFEF749F9A8F1E7
:1031D000006B4FEA9B25CBF34809C9F50074A74261
:1031E00000DC3C464DE04FF0006101EB85208A1485
:1031F0002849FFF7C9FF00260BE009EB0600254927
:1032000031F810004FF6FF71884200D003E0701CC7
:1032100086B2A642F1DB00BFA6421BDA4FF0006186
:1032200001EB8520FEF7B2F8002608E03AF8160018
:1032300006EB0901174A22F81100701C86B2A6425B
:10324000F4DB4FF0006101EB85208A14114900F096
:1032500023F804E022465146404600F01DF8A742FC
:1032600000D10FE06D1C4FF000090AEB440AA044A6
:10327000381B87B2B7F5007F02DD4FF4007400E021
:103280003C46B0E700BFFEF7C1F800BF9BE7000077
:1032900000000108CC0C00202DE9F04105460E4647
:1032A0001746002407E036F814102846FEF7B8F851
:1032B000AD1C601C84B2BC42F5DBBDE8F08110B5EA
:1032C00000F002F810BD00000CB500200190009045
:1032D0003348006840F480303149086000BF30480E
:1032E000006800F4003000900198401C01900098A4
:1032F00018B90198B0F5A06FF1D12948006800F421
:10330000003010B10120009001E0002000900098F2
:10331000012843D12348006840F01000214908608B
:103320000846006820F0030008600846006840F086
:10333000020008601A484068194948600846406819
:1033400048600846406840F480604860084640682D
:1033500020F47C1048600846406840F4E81048605B
:103360000846006840F08070086000BF0C480068A4
:1033700000F000700028F9D00948406820F00300F0
:10338000074948600846406840F00200486000BFB6
:103390000348406800F00C000828F9D10CBD00007B
:1033A0000010024000200240042808D14FF0E02124
:1033B000096941F004014FF0E022116107E04FF08C
:1033C000E021096921F004014FF0E022116170470A
:1033D00010B51348006840F0010011490860084624
:1033E0004068104908400E494860084600680E4988
:1033F00008400B4908600846006820F480200860F7
:103400000846406820F4FE0048604FF41F008860C2
:10341000FFF755FF4FF000600449086010BD000041
:10342000001002400000FFF8FFFFF6FE08ED00E08C
:1034300030B587B005460C4601210846FFF792F9E2
:10344000ADF81450ADF810400020ADF81600ADF8FE
:10345000120004A94FF0804000F048FB6020ADF856
:1034600000000120ADF802000920ADF8060002209E
:10347000ADF808006946400700F0E6FA0121880728
:1034800000F0ADFA0121880700F0B5FA07B030BDB1
:103490000EB50121FE4800F0BDFA00287ED0FFF7EE
:1034A000A3FC002002901BE29DF80800C0EBC000C6
:1034B000F84901EB8000407D01909DF80800062846
:1034C0006DDA9DF80400032869D1F34800780028DC
:1034D000FAD19DF8080008B9012000E000209DF80D
:1034E0000810012900D100E00021084338B1EB4861
:1034F00090F85F0008B1002000E0032000909DF8E4
:103500000800022801D1012000E000209DF80810E9
:10351000032901D1012100E00021084338B1DF482F
:1035200090F85F0008B1012000E0012000909DF8B4
:103530000800042801D1012000E000209DF80810B7
:10354000052901D1012100E00021084338B1D34809
:1035500090F85F0008B1032000E000200090CF4801
:1035600032309DF8001000EB81000068CB4991F8E3
:103570005A10C1F5967188420BDDC84890F85A0080
:10358000C0F59671C54832309DF8002000EB8200EE
:103590000160C24832309DF8001001E0B4E13BE028
:1035A00000EB81000168BD4890F85A00A0F59670C4
:1035B00081420BDAB94890F85A00A0F59670B749E5
:1035C00032319DF8002001EB820108609DF808006F
:1035D00000EBD0714910A0EB410161B9AF49323124
:1035E0009DF8002001EB82000168AC4A92F85A2055
:1035F000891A01600BE0A94932319DF8002001EBE6
:1036000082000168A54A92F85A20114401609DF891
:103610000800401CA24908709DF8080006287DDAC1
:103620009DF80400042879D19B4800780028FAD13D
:103630001D219DF80800C0EBC000964A02EB8000F7
:1036400041749DF8080008B9012000E000209DF8B1
:103650000810012900D100E00021084338B18F484B
:1036600090F85F0008B1002000E0032000909DF872
:103670000800022801D1012000E000209DF8081078
:10368000032901D1012100E00021084338B183481A
:1036900090F85F0008B1012000E0012000909DF843
:1036A0000800042801D1012000E000209DF8081046
:1036B000052901D1012100E00021084338B17748F4
:1036C00090F85F0008B1032000E0002000907348EC
:1036D00032309DF8001000EB810000686F4991F8CE
:1036E0005A10C1F5967188420BDD6C4890F85A006B
:1036F000C0F59671694832309DF8002000EB8200D9
:103700000160664832309DF8001000EB81000168CE
:10371000624890F85A00A0F5967000E033E08142CC
:103720000BDA5E4890F85A00A0F596705B4932318A
:103730009DF8002001EB820108609DF8080000EB75
:10374000D0714910A0EB410161B9544932319DF863
:10375000002001EB82000168504A92F85A20891A31
:1037600001600BE04D4932319DF8002001EB8200F1
:1037700001684A4A92F85A20114401609DF80800F5
:10378000401C474908709DF80800042814D19DF892
:103790000400042810D11D219DF80800C0EBC000D2
:1037A0003C4A02EB800041743B48007820B1012084
:1037B0003C4908800C2048809DF80800052814D159
:1037C0009DF80400042810D11D219DF80800C0EBCD
:1037D000C000304A02EB800041742F48007820B1CD
:1037E0000120304908800B2048809DF8080058B916
:1037F0009DF80400032807D12748007820B1012054
:10380000284908800A2048809DF8080002280BD12A
:103810009DF80400032807D11F48007820B101203B
:1038200020490880082048809DF8080003280BD113
:103830009DF80400032807D11748007820B1012023
:1038400018490880092048809DF8080004280BD1F9
:103850009DF80400032807D10F48007820B101200B
:10386000104908800C2048809DF8080005280BD1DD
:103870009DF80400032807D10748007820B10120F3
:10388000084908800B2048809DF8080006280BE0B6
:1038900000040040CC10002026000020A4150020C9
:1038A000220000201A00002008D19DF804000328FF
:1038B00004D1012015490880082048809DF808009F
:1038C000062808D19DF80400042804D101200F49DE
:1038D00008800A2048809DF80800401CC0B2029071
:1038E0009DF808000728FFF6DFAD09480068401C76
:1038F0000749086007480068401C06490860012124
:10390000054800F069F800BF0EBD00001A00002055
:10391000D40A0020D80A0020000400407FB50546E4
:103920000C4601210220FEF71DFFADF80850ADF84E
:1039300004400020ADF80600ADF80A00012211464F
:103940000C4800F078F801A90A4800F0CFF81D20D3
:103950008DF8000002208DF801008DF80200012092
:103960008DF803006846FEF747F90121014800F091
:1039700036F87FBD0004004010B50121124800F068
:1039800049F8F8B10121104800F026F80F48104915
:10399000098830F81100401E0B492C3108800D4871
:1039A000006808B9012000E000200A4908600848C2
:1039B0000088401C0649088008460088122801DB60
:1039C0000020088010BD000000080040E00A002030
:1039D000040B0020B4012242CA430282704721B185
:1039E000028842F00102028004E002884FF6FE7372
:1039F0001A400280704731B1B0F8442042F40042CE
:103A0000A0F8442005E0B0F84420C2F30E02A0F86C
:103A10004420704730B50246002000230024158A58
:103A200005EA0103958905EA010413B10CB10120EF
:103A300000E0002030BD1AB183890B43838102E08E
:103A400083898B438381704770B500240022002353
:103A5000058C4FF6EF7635400584028C8388048B05
:103A600048F6FF752C404FF6FF452C400D884FF669
:103A7000FF7606EA05252C434FF6DF752A400D89AF
:103A800006EA05152A434D8806EA05152A43154D11
:103A9000A84202D0144DA8421DD14FF67F752A408E
:103AA0004D894FF6FF7606EA05152A434FF6BF7596
:103AB0002A408D8806EA05152A434FF6FF352B402C
:103AC0004FF2FF752B408D8906EA85052B43CD8982
:103AD00006EA85052B4383800483CD88058702840D
:103AE00070BD0000002C014000340140002202881B
:103AF0001D4B98420ED01D4B98420BD0B0F1804F19
:103B000008D01B4B984205D01A4B984202D01A4B52
:103B1000984204D14FF68F731A404B881A43174BC3
:103B2000984207D0164B984204D04FF6FF431A40F4
:103B3000CB881A4302808B8883850B8803850A4BC8
:103B400098420BD0094B984208D00E4B984205D0B2
:103B50000D4B984202D00D4B984201D10B7A03864F
:103B60000123838270470000002C01400034014093
:103B70000004004000080040000C0040001000401D
:103B80000014004000400140004401400048014052
:103B900010B540F225511D4800F098F810B31B48AD
:103BA00000F050F9C4B21A48008800F40040C8B9C7
:103BB0001748008800F4804060B10A2C03D0002030
:103BC0001349088020E01248008840F40040104962
:103BD000088019E00D2C06D10D48008840F4804083
:103BE0000B49088010E00A480088C0F30D0009491D
:103BF0000C5407480088401C054908800846008886
:103C0000C72801DD0020088010BD000000380140F9
:103C100010000020300B002021B1828942F40052B4
:103C2000828104E082894DF6FF731A4082817047D9
:103C300010B504462048844209D101218803FEF7CB
:103C4000C1FD00214FF48040FEF7BCFD32E01B486F
:103C5000844209D101214804FEF794FD00214FF46C
:103C60000030FEF78FFD25E01548844209D101217F
:103C70008804FEF787FD00214FF48020FEF782FDC7
:103C800018E01048844209D10121C804FEF77AFDEA
:103C900000214FF40020FEF775FD0BE00A48844236
:103CA00008D101210805FEF76DFD00214FF48010B9
:103CB000FEF768FD10BD00000038014000440040E0
:103CC00000480040004C00400050004070B50246E3
:103CD000002400230025002040F66A16B14200D1DE
:103CE00000BFC1F3421501F01F03012606FA03F3DA
:103CF000012D02D19689334006E0022D02D1168AA9
:103D0000334001E0968A33400C12012606FA04F48F
:103D10001688344013B10CB1012000E0002070BDC2
:103D2000F0B50346002400260025002040F66A175F
:103D3000B94200D100BF1846C1F3421401F01F067A
:103D4000012707FA06F5012C01D10C3004E0022C02
:103D500001D1103000E014301AB107682F4307601A
:103D600002E00768AF430760F0BD00002DE9F047AF
:103D700086B005460E460024A24600BFA146002795
:103D8000B08900B100BF2F462C8A4CF6FF7004406A
:103D9000F08804432C82AC894EF6F3100440B088BE
:103DA00031890843718908430443AC81AC8A4FF6DA
:103DB000FF400440B0890443AC8201A8FEF718FD1F
:103DC0001F48874202D1DDF810A001E0DDF80CA009
:103DD000A88900F4004040B10AEBCA0000EB0A10C9
:103DE00031684900B0FBF1F807E00AEBCA0000EBCC
:103DF0000A1031688900B0FBF1F86420B8FBF0F0DC
:103E000004012009642101FB1089A88900F4004005
:103E100040B1322000EBC900B0FBF1F000F0070028
:103E2000044308E0322000EB09106421B0FBF1F0FC
:103E300000F00F0004432C8106B0BDE8F0870000BD
:103E40000038014001468888C0F308007047000030
:103E50002DE9F04105462C464FF480711248FDF7DC
:103E60003AFC00261CE0274607F08007802F04D18B
:103E7000B9000D48FDF731FC04E04FF400710A4829
:103E8000FDF729FC6006040E4FF480710648FDF72B
:103E900024FC4FF480710448FDF71DFC701CC6B271
:103EA000082EE0DBBDE8F081000C014010B50446AF
:103EB000FDF782FC7820FFF7CBFFFDF7A9FC00207F
:103EC000FFF7C6FFFDF7A4FC2046FFF7C1FFFDF793
:103ED0009FFCFDF789FC10BD10B50446FDF76CFC96
:103EE0007820FFF7B5FFFDF793FC4020FFF7B0FF08
:103EF000FDF78EFC2046FFF7ABFFFDF789FCFDF7D1
:103F000073FC10BD0FB4054B10B503A9044A029809
:103F100000F0EEF810BC5DF814FB0000294A000820
:103F20000C0000200FB4084B10B504A902AA039896
:103F300000F0DEF8044602A9002000F070FC2046E4
:103F400010BC5DF814FB00001F48000802E008C820
:103F5000121F08C1002AFAD170477047002001E003
:103F600001C1121F002AFBD1704700002DE9FF5F3D
:103F700082B00021DDE90430020DDDF840B00343DA
:103F800018D044F61050A2F2FF3242431514119893
:103F900001281FD0A5EB0B00401C5FEA000A4FF080
:103FA00000064E4FDFF83891B046504615D5CAF19D
:103FB000000413E0119801244AA3012801D16FEAFB
:103FC0000B010298119AC0E90031C0E9024206B023
:103FD000BDE8F09FCBF10000DFE704460021404A36
:103FE000491842EB0450CDE9001012E0E00707D079
:103FF00032463B4640464946FCF715FA804689461C
:1040000032463B4610461946FCF70DFA06460F4667
:104010006410002CEAD1DDE90401DDE90023BAF1E6
:10402000000F06DAFCF7FFF942464B46FCF7FBF9B6
:1040300005E0FCF76AFA42464B46FCF766FA04468E
:104040000E460022284BFCF7BDFC03D84FF0FF3092
:10405000014607E00022254B20463146FCF73CF99B
:10406000FCF798FC102409E0002C0ADB0A2200234C
:10407000FCF79AFB039B30321A55641E50EA01028A
:10408000F2D1641C039AC4F111031444119A012A59
:1040900003D0012208430DD10AE0084304D00020D8
:1040A0004FF0110B119072E7A3EB0B056D1E0DE0A5
:1040B0005B4504DD4FF0000205F1010504E003DA81
:1040C0004FF00002A5F10105002AECD002981199E9
:1040D000C0E90231C0E9004579E700000000144062
:1040E0000000F03F300000000000F0430000E03F1F
:1040F0002DE9FF4F95B09B468946064600250FE205
:10410000252877D100242746F84A0121059400E0AC
:10411000044316F8013F203B01FA03F01042F7D1A7
:1041200030782A2811D06FF02F033078A0F13002B8
:10413000092A16D8059A44F0020402EB820203EB26
:1041400042021044761C0590EFE759F8042B0592C3
:10415000002A03DA504244F40054059044F002046B
:10416000761C30782E2816D116F8010F44F004047E
:104170002A280DD06FF02F023078A0F13003092BE0
:1041800009D807EB870302EB4303C718761CF3E754
:1041900059F8047B761C30786C280FD006DC4C284C
:1041A00017D068280DD06A2814D104E0742810D0E4
:1041B0007A280FD10DE044F400140AE044F480148E
:1041C00001E044F440147278824202D104F5801474
:1041D000761C761C307866280BD013DC582877D0F4
:1041E00009DC002875D04528F6D04628F4D04728A9
:1041F0001AD19DE118E0632835D0642879D065286C
:1042000012D195E1702873D008DC6728F1D06928B5
:104210006FD06E280DD06F2806D1B5E073282CD052
:10422000752875D0782874D05A46179990476D1C18
:1042300075E1C4F30250022809D003280DD0D9F843
:10424000001004280DD00D6009F1040967E1D9F8C8
:104250000010EA17C1E90052F6E7D9F800100D8006
:10426000F2E70D70F0E719F8041B8DF8001000203C
:104270008DF80100EA46012003E059F804AB4FF045
:10428000FF3061074FF0000102D40DE008F1010199
:104290008846B9420FDA8045F8DB1AF80810002981
:1042A000F4D108E008F1010188468142FADB1AF8EE
:1042B00008100029F6D105985B46A0EB08072146B7
:1042C0003846179A00F094FA284400EB080507E0F6
:1042D0004DE029E10DE01AF8010B5A461799904775
:1042E000B8F10108F7D25B4621463846179A13E128
:1042F00042E00A220092C4F302524FF0000A022A5E
:1043000008D059F804CB032A4FEAEC710AD00DE02B
:1043100029E02AE009F1070121F00702F2E802C1D1
:10432000914609E00FFA8CFC4FEAEC71042A03D1A4
:104330004FFA8CFC4FEAEC71002907DA0A4600219B
:10434000DCF1000C61EB02012D2202E0220504D514
:104350002B228DF80420012203E0E20701D0202265
:10436000F7E7904659E00A2102E010220DE0102103
:104370004FF0000A00910BE010224FF0000A44F0C9
:1043800004040827009203E008224FF0000A00927C
:10439000C4F30252022A05D059F804CB0021032AA3
:1043A00008D009E009F1070121F00702F2E802C193
:1043B000914605E01FFA8CFC042A01D10CF0FF0C99
:1043C0004FF00008220728D5702806D0009B83F004
:1043D000100353EA0A0305D00EE040228DF80420B2
:1043E000012208E05CEA010206D030228DF80420A8
:1043F0008DF8050002229046009B83F0080353EAE3
:104400000A030AD15CEA010201D1620705D5302214
:104410008DF804204FF001087F1E582804D034A0E6
:1044200003900EA802900DE036A0F9E753466046CF
:10443000009AFCF7B9F984460398825C0298401E02
:10444000029002705CEA0100F0D1029806A9081AF5
:1044500000F1200A600702D524F4803400E001272F
:10446000574502DDA7EB0A0000E0002000EB0A013F
:10447000009005984144401A0590E00306D45B463D
:104480002146179A059800F0B3F90544002706E085
:1044900001A85A46C05D179990476D1C7F1C47457F
:1044A000F6DBE0030CD55B462146179A059800F031
:1044B0009FF9054404E030205A46179990476D1C37
:1044C0000099481E00900029F5DC08E00298029946
:1044D0005A460078491C0291179990476D1CBAF111
:1044E0000001AAF1010AF1DC65E1000009280100E0
:1044F000303132333435363738396162636465665A
:10450000000000003031323334353637383941421B
:10451000434445460000000000F058F90544761C6D
:10452000307800287FF4ECAD19B02846BDE8F08F54
:10453000620700D4062709F1070222F0070CFCE805
:104540000223E14603F000485FEA080C02D00FF2B4
:10455000702C0DE05FEA045C02D50FF2682C07E0D6
:104560005FEAC47C02D00FF2602C01E0AFF2700C65
:104570004FF0FF3823F00043CDF850C065280CD031
:1045800006DC452809D046281DD047283DD13DE00E
:10459000662818D067287ED138E00021112F01DB72
:1045A000112000E0781CCDE9000106A90EA8FFF754
:1045B000DDFCDDE90F010E9A03910021009207F165
:1045C000010A04914DE04FF000400097CDE9011041
:1045D00006A90EA8FFF7CAFCDDE90F0203920E9BA5
:1045E00011990022DDF80CA00093049211B9791CF6
:1045F00000EB010AB7EB0A0004D4C0F1FF3007F169
:10460000010A0490AAEB0700019044E0012F00DAB0
:1046100001270021112F01DD112000E03846CDE9EE
:10462000000106A90EA8FFF7A1FCDDE90F010E9A13
:104630000391002104910092BA4621070CD40399FA
:10464000514500DA8A46BAF1010F05DD009AAAF158
:104650000101515C302908D0B84202DA10F1040F90
:1046600006DA0121CDE9011015E0AAF10101E9E71F
:10467000002805DC049901440491AAEB000102E042
:10468000411C514500DD8A460499401A401C0190A6
:104690004FF000400290200704D40198504501DB00
:1046A000CDF8048000208DF84F0002980DF14F07DF
:1046B000B0F1004F25D02B200E9002984FF0020849
:1046C00000280CDA404202902D200E9007E00A21CB
:1046D0000298FCF753F83031029007F8011DB8F149
:1046E0000001A8F10108F2DC02980028EFD1791E40
:1046F0000E980870307800F0200040F0450007F870
:10470000020D12A8C01B00F107081498007800B130
:10471000012000EB0A01019801EBE071059841448A
:10472000401A401E0590E00306D45B462146179AC6
:10473000059800F05DF805441498007818B15A46C1
:10474000179990476D1CE00324D55B462146179AC4
:10475000059800F04DF805441CE00498002807DB9C
:10476000DDE90301884203DD0098405C179901E010
:10477000179930205A469047049805F10105401CCE
:1047800004900198401E019004D12E205A4617999A
:1047900090476D1CBAF10001AAF1010ADDDC05E0C9
:1047A00017F8010B5A46179990476D1CB8F1000194
:1047B000A8F10108F4DC5B462146179A0598ABE6A0
:1047C0002D0000002B000000200000002DE9F0412A
:1047D000044600251E461746880404D405E03946E1
:1047E0002020B0476D1C641EF9D52846BDE8F08135
:1047F0002DE9F041044600251E469046C80301D528
:10480000302700E02027880404D505E041463846DB
:10481000B0476D1C641EF9D52846BDE8F0810A68D2
:10482000531C0B601070704710B5044601200549F9
:104830000860204600F02CF800200349C1F8A801C8
:1048400010BD0000A80121420000214210B56FF008
:104850000400FEF7A9FD0A4800680A49B0FBF1F020
:10486000094908700846007800EB4001C1EBC01010
:104870004FF6FF7101EAC0000449088010BD000036
:10488000080B002000127A00080000200A00002017
:104890000146114A12884A434FF0E0235A61002230
:1048A0009A611A46126942F001021A6100BF4FF084
:1048B000E022106900F001021AB100F48032002AEF
:1048C000F5D04FF0E022126922F001024FF0E02310
:1048D0001A6100229A6170470A000020F8B500258D
:1048E000002600242F4800683221B0FBF1F084B28A
:1048F0004FF4616094FBF0F085B24FF4616094FB7B
:10490000F0F100FB11403C2190FBF1F086B23C201D
:1049100094FBF0F100FB114084B201200C237F22B4
:10492000014600905520FDF756FA0022052163202C
:10493000FDF7D8F9002208216320FDF7D3F9002202
:1049400005217220FDF7CEF9002208217220FDF723
:10495000C9F92A4614A11648FFF7E4FA00200C23EF
:10496000134A012100905620FDF75EFC32460EA14D
:104970000F48FFF7D7FA00200C230D4A01210090C1
:104980006520FDF751FC224607A10948FFF7CAFA46
:1049900000200C23064A012100907420FDF744FCFE
:1049A000F8BD0000D40A0020253032640000000069
:1049B000901100201FB501210820FDF7F3FE40F201
:1049C0000240ADF80C0004208DF80F0003208DF894
:1049D0000E0003A91348FCF7A1FD01210846FDF7CD
:1049E000E1FE01210846FCF779FD0220019000203C
:1049F0008DF8080008208DF8090001208DF80A00C4
:104A000001A8FCF779FC07208DF8000002208DF842
:104A1000010001208DF802008DF803006846FDF7C3
:104A2000EBF81FBD000C014000BF054A128802F0E0
:104A30004002002AF9D0C2B2014B1B1D1A807047F8
:104A40000038014030B589B005460C4600203F23B0
:104A5000102201460090FDF7BEF901201021CDE99A
:104A600000102807010E10232D4A0020FDF76EF9D3
:104A7000207810232BA2002100901846FDF7D4FBCC
:104A800029A103C9CDE907012078052307AA002140
:104A900000902020FDF764FB6078102324A21946C3
:104AA00000901846FDF7C0FB6078102321A219463C
:104AB00000902020FDF7B8FB1FA0006806906078EA
:104AC000032306AA102100903020FDF749FBA078AF
:104AD00010231AA2202100901846FDF7A5FB18A06C
:104AE00000680590A078042305AA202100900846BC
:104AF000FDF736FBE078102312A230210090184613
:104B0000FDF792FB10A103C9CDE90301E07805236D
:104B100003AA302100902020FDF722FB09B030BD10
:104B200046000020312E00000A0B0C060700000092
:104B3000322E0000562000000C060700332E000025
:104B40000D0E0607342E00000F100C0607000000A3
:104B50002DE9FC5F01200F213623FE4ACDE900102C
:104B600000210846FDF7F2F8FB4890F8630050B9C1
:104B700001200C210F23F94ACDE900100146332012
:104B8000FDF7E4F809E001200C210F23F44ACDE9F8
:104B9000001001463320FDF7D9F8EF4890F86A007D
:104BA000012809D10C211023EE4ACDE9001001465D
:104BB0004420FDF7CBF809E001200C211023EA4A3C
:104BC000CDE9001001464420FDF7C0F8FFF786FE4E
:104BD00003F0CEFAE04890F8620050B901201021AD
:104BE0003023E24ACDE9001027210B20FDF7AEF873
:104BF00018E0D94890F86200012809D1102130232B
:104C0000DB4ACDE9001027210B20FDF79FF809E0D2
:104C1000012010213023D74ACDE9001027210B2095
:104C2000FDF794F801201023D3A213210090462011
:104C3000FDF7FAFAD1480068FBF767FD05462A46FA
:104C40000B46CFA1D048FFF76DF901201023CE4AC3
:104C5000132100905020FDF7E7FA01201023CBA28A
:104C6000262100904620FDF7DFFA01201023C8A27C
:104C7000262100905020FDF7D7FA01203F2304227F
:104C80000F2100900020FDF7A6F800222721012027
:104C9000FDF728F8002227210320FDF723F8012043
:104CA0003F237F220F2100907B20FDF794F8002204
:104CB00027217C20FDF716F8002227217E20FDF712
:104CC00011F801203F233E223B2100900720FDF7F1
:104CD00082F801203F2378223B2100904120FDF7FC
:104CE0007AF89D4890F85F0000287DD000223C2192
:104CF0002320FCF7F7FF00223E212320FCF7F2FFE0
:104D000000223C215D20FCF7EDFF00223E215D20CA
:104D1000FCF7E8FF01203D2377221946009042204E
:104D2000FDF759F88C49D1F83200FBF76BFC82464D
:104D30000022994BFBF7E9FB07460022974BFBF754
:104D4000CBFA0546FBF7A9FC04460020A11CCAB219
:104D5000A11E0090C8B23D231946FDF73CF8012082
:104D60003E237D22102100901046FDF734F87A4949
:104D7000D1F83600FBF746FC8246894A894BFBF79F
:104D8000C4FB07460022884BFBF74AFB0546FBF7AE
:104D900084FC044600200090A01CC3B2A01EC1B237
:104DA0007D221046FDF717F880488088A0F57A70BC
:104DB000162190FBF1F01FFA80F900200090C9F154
:104DC0003E00C1B23E2302221046FDF704F8012046
:104DD0000090C9F13E00C3B2022210211046FCF738
:104DE000FAFF01203D2300E023E01A461946009017
:104DF0000720FCF7F0FF5849D1F83E00FBF702FC12
:104E000082460022644BFBF780FB07460022684B7A
:104E1000FBF762FA0546FBF740FC04460020A11CA4
:104E2000CAB2A11E0090C8B23D231946FCF7D3FFB9
:104E3000D2E000223C212220FCF754FF00223E2138
:104E40002220FCF74FFF00223C215D20FCF74AFFA7
:104E500000223E215D20FCF745FF01203D231A463C
:104E6000194600900720FCF7B6FF3B49D1F8320005
:104E7000FBF7C8FB05460022474BFBF746FB0746FE
:104E800000224C4BFBF728FA8246FBF706FC04464F
:104E90000020A11CCAB2A11E0090C8B23D23194631
:104EA000FCF799FF01203E230222102100901046BA
:104EB000FCF791FF2849D1F83600FBF7A3FB8246A7
:104EC000374A384BFBF721FB05460022364BFBF7F0
:104ED000A7FA0746FBF7E1FB044600200090A01C60
:104EE000C3B2A01EC1B202221046FCF774FF2F48C5
:104EF0008088A0F57A70162190FBF1F01FFA80F9F6
:104F000000200090C9F13E00C1B23E237D22104630
:104F1000FCF761FF01200090C9F13E00C3B27D2281
:104F200010211046FCF757FF01203D237722194638
:104F300000904220FCF74FFF0749D1F83E00FBF7F5
:104F400061FB07460022144BFBF7DFFA05460022FF
:104F5000124B31E09E000020A415002072010020B9
:104F6000040100209E010020B6010020160200204E
:104F700076020020D6020020540000001400002019
:104F800025312E3266560000280000205200000015
:104F900031322E36560000000000294000405740B4
:104FA00014AE47E17A942C4000804340BC0C0020B2
:104FB0000080414000004140FBF78EF98246FBF73C
:104FC0006CFB04460020A11CCAB2A11E0090C8B20E
:104FD0003D231946FCF7FFFEBDE8FC9F30B585B0C8
:104FE00005460C462078102344A200210090084674
:104FF000FDF71AF942A0006804902078042304AA5F
:10500000002100901020FDF7ABF8607810233DA23E
:10501000194600900020FDF707F93BA000680390B7
:105020006078042303AA102100900846FDF798F841
:10503000364890F8620088B9012D06D134480078CE
:1050400008B9012002E0002000E0012010230C221A
:10505000194600905820FDF711F827E02B4890F8EA
:105060006200012811D1012D06D12948007808B924
:10507000012002E0002000E0012010236E221946EA
:1050800000905820FCF7FAFF10E0012D06D12048CF
:10509000007808B9012002E0002000E00120102380
:1050A0006F22194600905820FCF7E8FFA0781023E3
:1050B00018A2202100900020FDF7B6F816A0006885
:1050C0000290A078042302AA202100901020FDF76E
:1050D00047F8E078102311A2302100900020FDF75E
:1050E000A3F80FA000680190E078042301AA302102
:1050F00000901020FDF734F805B030BD312E0000CF
:1051000015161112322E00001718191AA4150020B6
:1051100023000020332E00001B1C191A342E00001F
:10512000001D1E1F10B5044890F86400012802D12C
:105130000620FFF779FB10BDA41500202DE9F843E8
:10514000A0480078002873D19F480078012800D13A
:1051500000E000209C490978022901D1012100E0EA
:1051600000210843002856D0984890F85F0048B3C3
:1051700001203D237722194600904220FCF72BFEA8
:105180009249D1F83200FBF73DFA80460022904B5D
:10519000FBF7BBF9064600228E4BFBF79DF8044651
:1051A000FBF79AFA8C490880002000900978891C46
:1051B000CAB289490978891EC8B23D231946FCF74D
:1051C0000AFE28E001203D23772219460090422064
:1051D000FCF701FE7D49D1F83E00FBF713FA80464B
:1051E00000227B4BFBF791F906460022794BFBF737
:1051F00073F80446FBF770FA7749088000200090A6
:105200000978891CCAB274490978891EC8B23D233D
:105210001946FCF7E0FD6C480078032801D1012015
:1052200000E0002068490978042902D1012101E049
:10523000C3E00021084300284ED0644890F85F0086
:1052400050B301203E237D22102100901046FCF730
:10525000C2FD5E49D1F83600FBF7D4F906465F4A35
:105260005F4BFBF752F9044600225E4BFBF7D8F880
:105270008046FBF731FA5849088000200090084624
:105280000078801CC3B208460078801EC1B27D221F
:105290001046FCF7A0FD1FE0012038230222102158
:1052A00000901046FCF797FD4848D0F836000C21D6
:1052B00090FBF1F0C0F127004749088000200090E2
:1052C00008460078801CC3B208460078801EC1B230
:1052D00002221046FCF77FFD3B480078052801D1EB
:1052E000012000E0002038490978062901D1012178
:1052F00000E000210843002856D0344890F85F00B1
:1053000048B301203D231A46194600900720FCF7B8
:1053100062FD2E49D1F83E00FBF774F906460022E3
:105320002B4BFBF7F2F8044600222F4BFAF7D4FF81
:105330008046FBF7D1F928490880002000900978C1
:10534000891CCAB224490978891EC8B23D2319466E
:10535000FCF741FD28E001203D231A461946009044
:105360000720FCF738FD1949D1F83200FBF74AF95C
:1053700080460022164BFBF7C8F8064600221B4B5E
:10538000FAF7AAFF0446FBF7A7F9134908800020A3
:1053900000900978891CCAB20F490978891EC8B2E1
:1053A0003D231946FCF717FDFCF7BEFD10480068C9
:1053B00082B206490F48FDF7FBFE00200249087043
:1053C000BDE8F8832600002022000020A41500205C
:1053D00000002940004057400000002014AE47E183
:1053E0007A942C40008043400080414000004140BE
:1053F000DC0A002004FC000830B585B004460D46E8
:1054000001200F231F22002100900846FCF7E3FC37
:1054100020788DF8100060788DF81100A0788DF854
:105420001200E0788DF813000020042304AA01463E
:1054300000902020FCF794FE01200F237F22002102
:1054400000906020FCF7C7FC2878102329A2194699
:1054500000900020FCF7E8FE20798DF80C006079C0
:105460008DF80D00A0798DF80E00E0798DF80F0011
:105470002878042303AA102100900846FCF770FE48
:10548000687810231CA2202100900020FCF7CCFE9D
:10549000207A8DF80800607A8DF80900A07A8DF8DE
:1054A0000A00E07A8DF80B006878042302AA202114
:1054B00000901020FCF754FEA87810230FA2302192
:1054C00000900020FCF7B0FE207B8DF80400607B8C
:1054D0008DF80500A07B8DF80600E07B8DF80700B5
:1054E000A878042301AA302100901020FCF738FE90
:1054F00005B030BD312E0000322E0000332E0000EA
:105500007CB58F4890F86B00C0EB0010800000EB7A
:10551000C00101EB00108B490968B1EB400F49D97C
:10552000874890F86A00012844D1874800880521FF
:1055300090FBF1F201FB120090B91420FFF774F90F
:105540008248007878B901200C210F23804ACDE9E8
:10555000001001464420FCF7F9FBFCF7E5FC02E0F3
:105560001420FFF795F9784800880A2190FBF1F2A2
:1055700001FB120080B97548007868B901200C2140
:105580001023744ACDE9001001464420FCF7DEFBED
:10559000FFF7A4F9FCF7C8FC6B480088401C6A4977
:1055A000088008460088642804DD002065490860FA
:1055B0006549088068480088642190FBF1F201FB8E
:1055C000120000286AD161480078002866D1FFF7F0
:1055D00085F902F0CDFD61488088A0F57A7016212A
:1055E00090FBF1F05E490880554890F85F00C0B12B
:1055F0000020009008460088C0F13E00C1B23E2362
:1056000002221046FCF7E7FB012000905448008876
:10561000C0F13E00C3B2022210211046FCF7DBFBB2
:1056200017E0002000904E480088C0F13E00C1B253
:105630003E237D221046FCF7CEFB01200090484817
:105640000088C0F13E00C3B27D2210211046FCF755
:10565000C2FB414800884FF47A7190FBF1F201FBE4
:105660001200C8B93F480078012802D10A20FFF78C
:10567000DBF83D480068FBF748F8044622460B4635
:105680003AA13C48FEF74EFC01201023394A132171
:1056900000905020FCF7C8FDFCF746FC3648007827
:1056A000002803DDFFF73EFDFFF748FD274800789F
:1056B00041282CD102F0AEF8FCF736FC002024E0A3
:1056C0002E4931F810201E49223101EB4001098892
:1056D0008A4207DD294931F810201949223101EBAE
:1056E00040010A80254931F810201549891C01EB39
:1056F000400109888A4207DA204931F81020104910
:10570000891C01EB40010A80401C0428D8DB0F48AB
:1057100000782D2803D101F0C1F8FCF705FC1848EA
:10572000008818B1FFF7FEFC00F0F8F80748007891
:105730001449087008480088401C074908807CBD4F
:10574000A4150020D80A0020060000202600002012
:10575000880100209E01002004000020BC0C0020D5
:1057600002000020180000201400002025312E32F5
:10577000665600002800002022000020AC0C00200B
:105780001A0000202700002002F05AFC01E0FFF779
:10579000B7FEFCE7FEB507460C4615461E4601203F
:1057A0000F237F22002100900846FCF714FB002005
:1057B0003F237F2210210090FCF70DFB8DF808702D
:1057C0008DF809408DF80A508DF80B6000200423F5
:1057D00002AA014600902020FCF7C2FC01203F23D2
:1057E0007322102100901046FCF7F5FA01203F23A8
:1057F0007F22102100901046FCF7EDFA01200621CF
:105800000F23094ACDE9001010217420FCF79EFAFD
:10581000012006210F23054ACDE900103A2174200A
:10582000FCF794FAFEBD0000300000203B00002091
:105830002DE9FC5F06460F4614461D46DDF8308014
:1058400039462046FAF7D2FC294601904046FAF73D
:10585000CDFC834639463046FAF7C8FC59460090DD
:10586000FAF7CAFC82460199FAF7F8FC8146294604
:10587000FAF76AFCBDE8FC9F2DE9FC5F04460D4683
:1058800017461E46DDF83080B44200DD3446AC4297
:1058900000DA2C46BC4218DA3846FAF7A5FE8246F2
:1058A0002846FAF7A1FE83462046FAF79DFE0190AE
:1058B0001748184B5246594600900198FFF7B8FF19
:1058C0008146FAF7BDFE044617E03046FAF78CFE33
:1058D00082463846FAF788FE83462046FAF784FE69
:1058E00001900D480A4B5246594600900198FFF727
:1058F0009FFF8146FAF7A4FE0446B8F1000F04D0DA
:1059000040F6B830001BBDE8FC9F2046FBE70000D6
:105910000080BB4400007A440000FA442DE9F041C5
:10592000FCF7C2FCFE48007841281FD1FD480078F2
:1059300041281BD0002017E0FB4931F81020FB491B
:1059400001EB40010A80F84931F81020F749103185
:1059500001EB40010A80F44931F81020F34920316D
:1059600001EB40010A80401C0428E5DB002030E008
:10597000EE49303101EB80010968EC4A921E92F841
:105980005A20C2F5967291420ADDE849891E91F8C3
:105990005A10C1F59672E549303101EB80010A6079
:1059A000E249303101EB80010A68E049891E91F833
:1059B0005A10A1F596718A420ADADC49891E91F8DB
:1059C0005A10A1F59671D94A303202EB800211606B
:1059D000401C0428CCDBD64840880B287ED1D04818
:1059E00000780A280ED1D148801ED0F83200CF4965
:1059F000891E91F85A100844CC49891EC1F832001A
:105A000001F0B2FCC64800780B280ED1C748801EB2
:105A1000D0F83600C549891E91F85A100144C34890
:105A2000801EC0F8361001F0ADFCBD4800780C288F
:105A30000ED1BE48801ED0F83A00BC49891E91F8AC
:105A40005A100144B948801EC0F83A1001F0A8FC71
:105A5000B34800780D280ED1B448801ED0F83E001F
:105A6000B249891E91F85A100144B048801EC0F80E
:105A70003E1001F0A3FCAA4800780E280ED1AB48D6
:105A8000801ED0F84200A949891E91F85A1001449D
:105A9000A648801EC0F8421001F09EFCA048007885
:105AA0000F280ED1A148801ED0F846009F49891EBC
:105AB00091F85A1001449D48801EC0F8461001F02C
:105AC00099FC97480078102810D19848801ED0F88B
:105AD0004A009649891E91F85A1000E0DAE1014423
:105AE0009248801EC0F84A1001F092FC8C48007861
:105AF00011280ED18D48801ED0F84E008B49891E8A
:105B000091F85A1001448948801EC0F84E1001F0E7
:105B10008DFC8348007812280DD18448801E90F8AF
:105B2000520008B9012000E000208049891E81F858
:105B3000520001F055FD7A48007813280DD17B48BA
:105B4000801E90F8530008B9012100E00021774839
:105B5000801E80F8531001F051FD71480078142820
:105B60000DD17248801E90F8540008B9012100E060
:105B700000216E48801E80F8541001F04DFD6848E9
:105B8000007815280DD16948801E90F8550008B995
:105B9000012100E000216548801E80F8551001F0C9
:105BA00049FD5F48007816280DD16048801E90F8A6
:105BB000560008B9012100E000215C48801E80F8F1
:105BC000561001F045FD5648007817280DD157486A
:105BD000801E90F8570008B9012100E000215348C9
:105BE000801E80F8571001F041FD4D4800781828BC
:105BF0000DD14E48801E90F8580008B9012100E0F0
:105C000000214A48801E80F8581001F03DFD4448AC
:105C1000007819280DD14548801E90F8590008B920
:105C2000012100E000214148801E80F8591001F058
:105C300039FD3B4800783D280DD13C48801E90F846
:105C40005F0008B9012000E000203849891E81F872
:105C50005F0001F049FF3248007837280AD1334805
:105C6000801EB0F86000401C3049891EA1F8600019
:105C700000F07EFE2A480078382813D12B49891E6F
:105C8000D1F85B00FAF741FD06462A4A2A4BFAF79B
:105C900023FB0446FAF74CFD2449891EC1F85B003A
:105CA00000F02AFD1E480078392813D11F49891EAB
:105CB000D1F86600FAF729FD0646204A204BFAF78C
:105CC0000BFB0446FAF734FD1849891EC1F866003B
:105CD00001F006F812480078342812D11348801ECB
:105CE00090F85A00401C1149891E81F85A00084654
:105CF00090F85A00092802DD092081F85A0001F0C5
:105D0000F7FC074800781F2825D10848801E90F826
:105D10006200401C0549891E81F86200084611E0B6
:105D20002600002027000020AC0C0020A615002033
:105D30001A0000207B14AE47E17A843F9A99999922
:105D40009999B93F90F86200022802DD002081F89D
:105D5000620001F0BDFEFE48007823280BD1FD480B
:105D600090F8630008B9012000E00020F94981F8AB
:105D7000630001F015FDF648007822280BD1F548A4
:105D800090F86E0008B9012000E00020F14981F888
:105D90006E0001F01FFAEE48007835280BD1ED486F
:105DA00090F8640008B9012000E00020E94981F87A
:105DB000640000F037FCE648007836280BD1E5484F
:105DC00090F8650008B9012000E00020E14981F861
:105DD000650001F01DF8DE4800783A280BD1DD4857
:105DE00090F86A0008B9012000E00020D94981F844
:105DF0006A0001F0DBF8D64800783B2810D1D5487E
:105E000090F86B00401CD34981F86B00084690F86D
:105E10006B003C2802DD3C2081F86B0001F03CF96E
:105E2000CB4800783C280BD1CA4890F86C0008B9E0
:105E3000012000E00020C74981F86C0001F040F823
:105E4000C34800783F2810D1C24890F86D00401D2B
:105E5000C04981F86D00084690F86D00642802DDA5
:105E6000642081F86D0001F0FBF9B948007824281E
:105E700010D1B84890F86F00801CB64981F86F00C7
:105E8000084690F86F000F2802DD0F2081F86F00A0
:105E900000F006FEB04840880C287CD1AC48007861
:105EA0000A280BD1AB48D0F83200AA4991F85A1011
:105EB000401AA849C1F8320001F056FAA448007807
:105EC0000B280BD1A348D0F83600A24991F85A10FC
:105ED000411AA048C0F8361001F054FA9C480078E6
:105EE0000C280BD19B48D0F83A009A4991F85A10E7
:105EF000411A9848C0F83A1001F052FA94480078D4
:105F00000D280BD19348D0F83E00924991F85A10D1
:105F1000411A9048C0F83E1001F050FA8C480078C1
:105F20000E280BD18B48D0F842008A4991F85A10BC
:105F3000411A8848C0F8421001F04EFA84480078AF
:105F40000F280BD18348D0F84600824991F85A10A7
:105F5000411A8048C0F8461001F04CFA7C4800789D
:105F600010280BD17B48D0F84A007A4991F85A1092
:105F7000411A7848C0F84A1001F04AFA744800788B
:105F800011280DD17348D0F84E00724991F85A107B
:105F9000411A704800E0A6E1C0F84E1001F046FA40
:105FA0006B48007812280BD16A4890F8520008B963
:105FB000012000E00020674981F8520001F010FB49
:105FC0006348007813280BD1624890F8530008B951
:105FD000012100E000215F4880F8531001F00EFB22
:105FE0005B48007814280BD15A4890F8540008B93F
:105FF000012100E00021574880F8541001F00CFB0B
:106000005348007815280BD1524890F8550008B92C
:10601000012100E000214F4880F8551001F00AFBF3
:106020004B48007816280BD14A4890F8560008B91A
:10603000012100E00021474880F8561001F008FBDC
:106040004348007817280BD1424890F8570008B908
:10605000012100E000213F4880F8571001F006FBC5
:106060003B48007818280BD13A4890F8580008B9F6
:10607000012100E00021374880F8581001F004FBAE
:106080003348007819280BD1324890F8590008B9E4
:10609000012100E000212F4880F8591001F002FB97
:1060A0002B4800783D280BD12A4890F85F0008B9AA
:1060B000012000E00020274981F85F0001F014FD75
:1060C00023480078372808D12248B0F86000401EE5
:1060D0002049A1F8600000F04BFC1D4800783828EA
:1060E00011D11C49D1F85B00FAF70FFB06461B4A99
:1060F0001B4BFAF792F90446FAF71AFB1549C1F857
:106100005B0000F0F9FA12480078392811D11149E2
:10611000D1F86600FAF7F9FA0646124A124BFAF776
:106120007CF90446FAF704FB0A49C1F8660000F05E
:10613000D7FD0748007834281FD1064890F85A0048
:10614000401E044981F85A00084690F85A000DE0B4
:1061500026000020A41500201A0000207B14AE4762
:10616000E17A843F9A9999999999B93F012802DA7D
:10617000012081F85A0001F0BBFAC54800781F28B9
:1061800011D1C44890F8620020B90220C14981F8B9
:10619000620006E0BF4890F86200401EBD4981F8E9
:1061A000620001F095FCBA48007823280BD1B94869
:1061B00090F8630008B9012000E00020B54981F89B
:1061C000630001F0EDFAB248007822280BD1B14803
:1061D00090F86E0008B9012000E00020AD4981F878
:1061E0006E0000F0F7FFAA48007835280BD1A948C7
:1061F00090F8640008B9012000E00020A54981F86A
:10620000640000F00FFAA248007836280BD1A148AC
:1062100090F8650008B9012000E000209D4981F850
:10622000650000F0F5FD9A4800783A280BD19948AE
:1062300090F86A0008B9012000E00020954981F833
:106240006A0000F0B3FE924800783B2810D19148D4
:1062500090F86B00401E8F4981F86B00084690F85B
:106260006B00012802DA012081F86B0000F014FFB6
:10627000874800783C280BD1864890F86C0008B914
:10628000012000E00020834981F86C0000F018FE36
:106290007F4800783F2811D17E4890F86D0005288E
:1062A00003DA05207B4981F86D007A4890F86D008B
:1062B000401F784981F86D0000F0D2FF74480078E3
:1062C000242810D1734890F86F00801E714981F81E
:1062D0006F00084690F86F000B2802DA0B2081F857
:1062E0006F0000F0DDFB6C48408808287ED16848CC
:1062F00000780A2801D101F037F8654800780B28AA
:1063000001D101F03FF8624800780C2801D101F07A
:1063100047F85F4800780D2801D101F04FF85C483C
:1063200000780E2801D101F057F8594800780F285D
:1063300001D101F05FF856480078102801D101F032
:1063400067F853480078112801D101F06FF85048E0
:106350000078122801D101F043F94D480078132844
:1063600001D101F04BF94A480078142801D101F01D
:1063700053F947480078152801D101F05BF94448EA
:106380000078162801D101F063F9414800781728F8
:1063900001D101F06BF93E480078182801D101F0D5
:1063A00073F93B480078192801D101F07BF938488E
:1063B00000783D2801D101F097FB35480078372857
:1063C00001D100F0D5FA32480078382801D100F028
:1063D00093F92F480078342801D101F089F92C482D
:1063E00000781F2801D101F073FB00E03BE0284852
:1063F0000078232801D101F0D3F92548007822281C
:1064000001D100F0E7FE22480078352801D100F0E4
:1064100009F91F480078362801D100F0F9FC1C4822
:1064200000783A2801D100F0C1FD194800783B28D6
:1064300001D100F031FE164800783C2801D100F06F
:106440003FFD13480078392801D100F049FC10487D
:1064500000783F2801D100F003FF0D480078242880
:1064600001D100F01DFB0A4800780C4909788842E8
:1064700006D00B48006882B206490A48FCF798FE2D
:10648000FBF752FD002004490880BDE8F0810000C0
:1064900026000020A41500201A000020270000205C
:1064A000DC0A002004FC000808B5FBF707FC01200B
:1064B0003F234022002100901846FBF78CFC08BDCA
:1064C00008B5FBF7FBFB01203F2340220021009091
:1064D0001846FBF780FC08BD08B5FBF7EFFB012071
:1064E0003F234022002100901846FBF774FC08BDB2
:1064F0002DE9F04F85B006460D4691461F46DDE971
:106500000F4800203F23102211460090FBF763FC48
:10651000701E032190FBF1F201FB1200000110300C
:1065200000F0FF0A012010210B463D4ACDE9001082
:1065300051460020FBF70AFC287810234A461946EA
:1065400000901846FBF770FE20788DF810006078F8
:106550008DF81100A0788DF81200E0788DF8130006
:106560002878042304AA102100902020FBF7F8FDCE
:10657000687810233A46202100901846FBF754FE15
:1065800020798DF80C0060798DF80D00A0798DF8D8
:106590000E00E0798DF80F006878042303AA20210B
:1065A00000900846FBF7DCFDA8781023009030210E
:1065B00018460E9AFBF738FE207A8DF80800607AAC
:1065C0008DF80900A07A8DF80A00E07A8DF80B00AA
:1065D000A878042302AA302100902020FBF7C0FDF8
:1065E000002039237E22162100907420FBF7F3FB54
:1065F000700190FBF8F0183000F0FF0A700190FB7A
:10660000F8F0133000F0FF0B012053467E2259466C
:1066100000907420FBF7DFFB05B0BDE8F08F0000B1
:106620004600002000B587B024A30FCBCDE9052399
:10663000CDE9030125A00068029002A903A8FEF796
:10664000DBFE01201021CDE90010214890F85A20EE
:1066500001235820FBF79EFD1D4890F86400012897
:106660000FD11C48007808B9012000E000200E215D
:106670001023194ACDE9001021215820FBF766FBB1
:106680000EE01448007808B9012000E000200E2137
:106690001023124ACDE9001021215820FBF756FBA8
:1066A00001201021CDE90010094890F86520012350
:1066B00030215820FBF76EFD07B000BD36370809C2
:1066C00002034445464748492E4A4B4C010001000D
:1066D000A415002023000020660000208200002076
:1066E00008B504A00068009069460220FEF776FC19
:1066F00008BD00000101000130B587B026A30FCB13
:1067000003AC0FC428A00068029002A903A8FEF7FA
:1067100073FE26480068F9F7F8FF044622460B4648
:1067200023A12548FDF7FEFB01201023224A19462C
:1067300000905820FBF778FD2049D1F85B00F9F76D
:10674000E4FF044622460B4619A11B48FDF7EAFB6D
:106750001B48007808B9012000E000201023164AE9
:10676000202100905820FBF75FFD1449D1F8660006
:10677000F9F7CBFF044622460B4612A10E48FDF75F
:10678000D1FB012010230C4A302100905820FBF748
:106790004BFD07B030BD00005051080950513E3F3D
:1067A000383950511112383901000100140000200D
:1067B00025312E326656000028000020A415002046
:1067C0002300002025322E316656000008B504A0B3
:1067D0000068009069460220FEF734F908BD000009
:1067E0000101000100B58BB00EA000680A900EA058
:1067F000006809900DA0006808900DA0006807903F
:106800000CA207CA04AB07C3062004A907AA08AB59
:10681000CDE90021029009AA0AA90120FFF768FE2C
:106820000BB000BD00010100312E0000322E00002F
:10683000332E000036370809505108095253080911
:1068400000B58BB00EA000680A900EA000680990F9
:106850000DA0006808900DA0006807900CA207CA60
:1068600004AB07C3092004A907AA08ABCDE900219E
:10687000029009AA0AA90720FFF73AFE0BB000BD53
:1068800000010100372E0000382E0000392E0000D4
:1068900030313233343508092F436B4A2DE9F84340
:1068A000002455E02C4901EB8401096801F5FA60E8
:1068B000F9F79AFE0746284901EB8401096801F5BA
:1068C0007A70F9F791FE8046244931F81400F9F7FF
:1068D00094FE8146224800233A46414600904846AD
:1068E000FEF7A6FF0646F9F7C4FEC5B21D480078BC
:1068F0001D490978884201D0012000E000201B4991
:10690000095DA94201D0012100E000210843E8B15E
:10691000012023010C33DAB2C5F13F03D9B22301C0
:106920001B1D0090D8B23F23FBF755FA0020C5F19C
:106930003F01CBB221010C31CAB22101091D0090E7
:10694000C8B20021FBF747FA08480555601CC4B2DD
:10695000082CA7DBBDE8F883D6150020BC0C00206E
:1069600000007C4226000020270000207406002042
:1069700030B587B026A30FCB03AC0FC428A00068A6
:10698000029002A903A8FEF737FD26480068F9F730
:10699000BCFE044622460B4623A12548FDF7C2FA59
:1069A0002448007808B9012000E000201023204A84
:1069B000194600905820FBF737FC1F49D1F85B00BF
:1069C000F9F7A3FE044622460B4617A11848FDF727
:1069D000A9FA01201023164A202100905820FBF725
:1069E00023FC1549D1F86600F9F78FFE04462246CC
:1069F0000B4612A10E48FDF795FA012010230C4A10
:106A0000302100905820FBF70FFC07B030BD00008C
:106A10005051080950513E3F383950511112383900
:106A2000000101001400002025312E3266560000BE
:106A30002800002023000020A415002025322E313C
:106A40006656000000B58BB00EA000680A900EA03C
:106A5000006809900DA0006808900DA000680790DC
:106A60000CA207CA04AB07C3062004A907AA08ABF7
:106A7000CDE90021029009AA0AA90220FFF738FDFA
:106A80000BB000BD01000100312E0000322E0000CD
:106A9000332E0000363708095051080952530809AF
:106AA00008B504A0006800906946022001F05AF978
:106AB00008BD00000101000000B58BB00EA0006809
:106AC0000A900EA0006809900DA0006808900DA023
:106AD000006807900CA207CA04AB07C3092004A9E9
:106AE00007AA08ABCDE90021029009AA0AA9FFF77D
:106AF000FFFC0BB000BD000001010000372E0000BC
:106B0000382E0000392E0000303132333435080978
:106B10002F436B4A1CB5FBF7D1F80120102311A2BB
:106B2000002100900846FBF77FFB10A00068019051
:106B30000120042301AA002100902820FBF710FB6C
:106B4000012010230AA2194600900020FBF76CFBDD
:106B50000120102309A2202100900020FBF764FBF4
:106B60001CBD00004A323052430000002E256869E7
:106B7000323032302E31322E32300000322E32009E
:106B800000B58BB00EA000680A900EA000680990B6
:106B90000DA0006808900DA0006807900CA207CA1D
:106BA00004AB07C3062004A907AA08ABCDE900215E
:106BB000029009AA0AA9FFF79BFC0BB000BD0000D8
:106BC00001010000342E0000352E0000362E00009A
:106BD0003A3B08093C3D3E3F404166671FB5FBF725
:106BE0006DF814A103C9CDE902010120072302AA0F
:106BF000102100900020FBF7B3FA01201023462259
:106C0000202100900020FBF739FA012010230BA26D
:106C1000202100901846FBF707FB0AA000680190AE
:106C20000120022301AA202100903820FBF798FAC6
:106C30001FBD00005E40416667080900456E74652F
:106C400072000000646500001CB5FBF737F806A071
:106C5000006801900120042301AA1821009020203F
:106C6000FBF77EFA1CBD000040416C2700B58BB0DD
:106C70000EA000680A900EA0006809900DA00068A0
:106C800008900DA0006807900CA207CA04AB07C3C8
:106C9000092004A907AA08ABCDE90021029009AA9E
:106CA0000AA90320FFF724FC0BB000BD010100007E
:106CB000312E0000322E0000332E000000010203AE
:106CC000000104050607080908B504A00068009043
:106CD00069460320FDF7B6FE08BD00000101010072
:106CE00030B587B026A30FCB03AC0FC428A0006833
:106CF000029002A903A8FEF77FFB26480068F9F777
:106D000004FD044622460B4623A12548FDF70AF957
:106D100001201023224A194600905820FBF784FADC
:106D20002049D1F85B00F9F7F0FC044622460B46F7
:106D300019A11B48FDF7F6F801201023184A20215D
:106D400000905820FBF770FA1649D1F86600F9F761
:106D5000DCFC044622460B4613A11148FDF7E2F87D
:106D60001348007808B9012000E0002010230C4AE5
:106D7000302100905820FBF757FA07B030BD0000D3
:106D80005051080950513E3F38395051111238398D
:106D9000010100001400002025312E32665600004B
:106DA00028000020A415002025322E316656000050
:106DB0002300002000B58BB00EA000680A900EA042
:106DC000006809900DA0006808900DA00068079069
:106DD0000CA207CA04AB07C3092004A907AA08AB81
:106DE000CDE90021029009AA0AA90420FFF780FB3F
:106DF0000BB000BD00010100342E0000352E000054
:106E0000362E000011121314202108090001292632
:106E100000B587B021A30FCBCDE90523CDE9030150
:106E200022A00068029002A903A8FEF7E5FA01205B
:106E30001021CDE900101E4890F85A200123582057
:106E4000FBF7A8F91A4890F86400012809D10E212F
:106E50001023184ACDE9001021215820FAF776FFB7
:106E600009E001200E211023134ACDE90010212151
:106E70005820FAF76BFF1148007808B9012000E0AC
:106E800000201021CDE90010094890F86520012369
:106E900030215820FBF77EF907B000BD36370809CE
:106EA00002034445464748492E4A4B4C0101000025
:106EB000A41500206600002082000020230000208E
:106EC00000B587B02DA30FCBCDE90523CDE9030194
:106ED0002EA00068029002A903A8FEF78DFA2C48A4
:106EE00090F86A00012809D10E211023294ACDE922
:106EF000001011215820FAF729FF09E001200E2186
:106F00001023254ACDE9001011215820FAF71EFF61
:106F10001F4890F86B2021A12248FDF703F80120BB
:106F20001023204A202100905820FBF77DF91848B3
:106F300090F86C0001280FD11B48007808B9012097
:106F400000E000200E211023124ACDE9001031216B
:106F50005820FAF7FBFE0EE01348007808B901202C
:106F600000E000200E2110230B4ACDE90010312152
:106F70005820FAF7EBFE07B000BD00005253080995
:106F800052533839525354552E4A5B5C010100006C
:106F9000A415002066000020820000202530326405
:106FA0006D696E00901100202300002000B587B0AD
:106FB0002DA30FCBCDE90523CDE903012EA0006859
:106FC000029002A903A8FEF717FA2C4890F86A006D
:106FD00001280FD12A48007808B9012000E00020DC
:106FE0000E211023274ACDE9001011215820FAF76D
:106FF000ADFE0EE02248007808B9012000E0002034
:107000000E211023204ACDE9001011215820FAF753
:107010009DFE1A4890F86B201CA11E48FCF782FFC9
:10702000012010231B4A202100905820FBF7FCF878
:10703000124890F86C00012809D10E211023114A42
:10704000CDE9001031215820FAF780FE09E0012037
:107050000E2110230C4ACDE9001031215820FAF7F7
:1070600075FE07B000BD000052530809525338396D
:10707000525354552E4A5B5C00010100A4150020B8
:1070800023000020660000208200002025303264AA
:107090006D696E009011002000B587B02AA30FCB58
:1070A000CDE90523CDE903012BA00068029002A9D8
:1070B00003A8FEF7A1F9294890F86A00012809D130
:1070C0000E211023264ACDE9001011215820FAF78D
:1070D0003DFE09E001200E211023224ACDE90010D7
:1070E00011215820FAF732FE1C4890F86B201EA19F
:1070F0001F48FCF717FF1F48007808B9012000E07F
:10710000002010231A4A202100905820FBF78CF809
:10711000124890F86C00012809D10E211023104A62
:10712000CDE9001031215820FAF710FE09E00120C6
:107130000E2110230B4ACDE9001031215820FAF717
:1071400005FE07B000BD00005253080952533839FC
:10715000525354552E4A5B5C01000100A4150020D7
:107160006600002082000020253032646D696E00C8
:10717000901100202300002000B58BB00EA0006805
:107180000A900EA0006809900DA0006808900DA05C
:10719000006807900CA207CA04AB07C3062004A925
:1071A00007AA08ABCDE90021029009AA0AA9032089
:1071B000FFF79EF90BB000BD01010000312E000069
:1071C000322E0000332E00003637080950510809CE
:1071D0005253080908B504A00068009069460020D1
:1071E00000F0C0FD08BD00000001010000B58BB03B
:1071F0000EA000680A900EA0006809900DA000681B
:1072000008900DA0006807900CA207CA04AB07C342
:10721000092004A907AA08ABCDE90021029009AA18
:107220000AA90520FFF764F90BB000BD01000100B9
:10723000342E0000352E0000362E000011121314DB
:10724000202108090001292608B504A00068009043
:1072500069460020FDF7F6FB08BD000000010101B2
:1072600000B587B01FA30FCBCDE90523CDE90301FE
:1072700020A00068029002A903A8FEF7BDF81E48EE
:1072800090F85F0040B1012010232A221946009097
:107290005820FAF7F3FE07E0012010232B221946AD
:1072A00000905820FAF7EAFE012010236D221946BB
:1072B00000906820FAF7E2FE0F4890F86D200FA1C9
:1072C0001048FCF72FFE1048007808B9012000E0B4
:1072D000002010230B4A302100905820FAF7A4FF19
:1072E00007B000BD3A3B08093A3B56573A3B582491
:1072F00059071B5A01010000A415002025303364F2
:1073000025250000901100202300002000B58BB03F
:107310000EA000680A900EA0006809900DA00068F9
:1073200008900DA0006807900CA207CA04AB07C321
:10733000092004A907AA08ABCDE90021029009AAF7
:107340000AA90120FFF7D4F80BB000BD000101002D
:10735000312E0000322E0000332E00000001020307
:1073600000010405060708091CB504A103C9CDE9FD
:1073700000010121684600F049FF1CBD0001010128
:10738000010101011CB504A103C9CDE900010221DD
:10739000684600F03BFF1CBD010001010101010135
:1073A0001CB504A103C9CDE900010321684600F022
:1073B0002DFF1CBD01010001010101011CB504A14B
:1073C00003C9CDE900010421684600F01FFF1CBD80
:1073D00001010100010101011CB504A103C9CDE9AE
:1073E00000010521684600F011FF1CBD01010101EB
:1073F000000101011CB504A103C9CDE9000106216A
:10740000684600F003FF1CBD0101010101000101FC
:107410001CB504A103C9CDE900010721684600F0AD
:10742000F5FE1CBD01010101010100011CB504A113
:1074300003C9CDE900010821684600F0E7FE1CBD44
:10744000010101010101010000B58BB00EA000682F
:107450000A900EA0006809900DA0006808900DA089
:10746000006807900CA207CA04AB07C3092004A94F
:1074700007AA08ABCDE90021029009AA0AA90620B3
:10748000FFF736F80BB000BD01010000342E0000FC
:10749000352E0000362E0000111213142021080989
:1074A000000129261CB504A103C9CDE90001012171
:1074B000684601F01FF91CBD000101010101010135
:1074C0001CB504A103C9CDE900010221684601F001
:1074D00011F91CBD01000101010101011CB504A14C
:1074E00003C9CDE900010321684601F003F91CBD81
:1074F00001010001010101011CB504A103C9CDE98D
:1075000000010421684601F0F5F81CBD01010100ED
:10751000010101011CB504A103C9CDE90001052148
:10752000684601F0E7F81CBD0101010100010101FD
:107530001CB504A103C9CDE900010621684601F08C
:10754000D9F81CBD01010101010001011CB504A114
:1075500003C9CDE900010721684601F0CBF81CBD45
:1075600001010101010100011CB504A103C9CDE91C
:1075700000010821684601F0BDF81CBD01010101B0
:107580000101010000B58BB00EA000680A900EA0AA
:10759000006809900DA0006808900DA00068079091
:1075A0000CA207CA04AB07C3092004A907AA08ABA9
:1075B000CDE90021029009AA0AA90220FEF798FF4E
:1075C0000BB000BD01000100312E0000322E000082
:1075D000332E00000001020300010405060708091C
:1075E0001CB504A103C9CDE900010121684601F0E1
:1075F0006FF91CBD00010101010101011CB504A1CD
:1076000003C9CDE900010221684601F061F91CBD02
:1076100001000101010101011CB504A103C9CDE96B
:1076200000010321684601F053F91CBD010100016E
:10763000010101011CB504A103C9CDE90001042128
:10764000684601F045F91CBD01010100010101017D
:107650001CB504A103C9CDE900010521684601F06C
:1076600037F91CBD01010101000101011CB504A194
:1076700003C9CDE900010621684601F029F91CBDC6
:1076800001010101010001011CB504A103C9CDE9FB
:1076900000010721684601F01BF91CBD0101010131
:1076A000010100011CB504A103C9CDE900010821B5
:1076B000684601F00DF91CBD010101010101010045
:1076C00008B504A00068009069460320FDF786FC19
:1076D00008BD00000101010008B504A00068009089
:1076E00069460120FDF7AEF908BD00000100010167
:1076F00000B587B021A30FCBCDE90523CDE9030168
:1077000022A00068029002A903A8FDF775FE204898
:10771000007808B9012000E000201021CDE9001018
:107720001C4890F85A2001235820FAF733FD1948D5
:1077300090F86400012809D10E211023164ACDE9E2
:10774000001021215820FAF701FB09E001200E2149
:107750001023124ACDE9001021215820FAF7F6FA39
:1077600001201021CDE900100A4890F8652001237E
:1077700030215820FAF70EFD07B000BD3637080952
:1077800002034445464748492E4A4B4C000101003C
:1077900023000020A41500206600002082000020A5
:1077A00008B504A0006800906946012000F0DAFAEC
:1077B00008BD00000100010000B58BB00EA00068FC
:1077C0000A900EA0006809900DA0006808900DA016
:1077D000006807900CA207CA04AB07C3062004A9DF
:1077E00007AA08ABCDE90021029009AA0AA9052041
:1077F000FEF77EFE0BB000BD01000100342E00003C
:10780000352E0000362E00003A3B08093C3D3E3F35
:10781000404166671CB50120102350A20021009052
:107820000220FAF701FD01201021CDE900104C489B
:107830004288042300211220FAF7ACFC0120102119
:10784000CDE900104648428A042300213820FAF787
:10785000A1FC01201021CDE900104148428C0423F5
:1078600000215F20FAF796FC012010233DA2194663
:1078700000900220FAF7D8FC01201021CDE9001079
:107880003748828804231220FAF784FC0120102153
:10789000CDE900103248828A04233820FAF77AFCB6
:1078A00001201021CDE900102D48828C04235F2097
:1078B000FAF770FC012010232BA220210090022057
:1078C000FAF7B2FC01201021CDE900102448C2884B
:1078D000042320211220FAF75DFC01201021CDE9BC
:1078E00000101F48C28A042320213820FAF752FCD6
:1078F00001201021CDE900101948C28C0423202159
:107900005F20FAF747FC0120102318A230210090D5
:107910000220FAF789FC01201021CDE9001010485F
:107920000289042330211220FAF734FC01201021AF
:10793000CDE900100A48028B042330213820FAF7E1
:1079400029FC01201021CDE900100548028D0423F7
:1079500030215F20FAF71EFC1CBD0000313A000008
:10796000A4150020323A0000333A0000343A0000F7
:1079700000B589B0FAF7A2F9012010232BA200214B
:1079800000900846FAF750FC29A103C9CDE9070188
:107990000120062307AA002100901020FAF7E0FB3F
:1079A0000120102324A2002100907020FAF73CFC53
:1079B00022A103C9CDE905010120062305AA102152
:1079C00000900846FAF7CCFB012010231DA22021CD
:1079D00000900020FAF728FC1BA103C9CDE90301A0
:1079E0000120072303AA202100901020FAF7B8FBFA
:1079F000012010234622302100900020FAF73EFBA0
:107A00000120102312A2302100901846FAF70CFC36
:107A100011A0006802900120022302AA30210090E8
:107A20003820FAF79DFB09B000BD0000312E0000A0
:107A30005D5E2C2D5F6000002C00000061623A3B0F
:107A400000010000322E00005D5E11124A635000FA
:107A5000456E7465720000006465000008B504A0FE
:107A60000068009069460020FDF7B8FA08BD0000E4
:107A70000001010100B58BB00EA000680A900EA0B5
:107A8000006809900DA0006808900DA0006807909C
:107A90000CA207CA04AB07C3092004A907AA08ABB4
:107AA000CDE90021029009AA0AA90820FEF720FDCD
:107AB0000BB000BD01000100372E0000382E000081
:107AC000392E000030313233343508092F436B4AE8
:107AD00008B504A00068009069460120FDF77EFA11
:107AE00008BD00000100010100B587B024A30FCB41
:107AF000CDE90523CDE9030125A00068029002A984
:107B000003A8FDF779FC234890F85F0068B122488C
:107B1000007808B9012000E0002010232A2219462D
:107B200000905820FAF7AAFA0CE01B48007808B930
:107B3000012000E0002010232B221946009058203D
:107B4000FAF79CFA1448007808B9012000E00020F8
:107B500010236D22194600906820FAF78FFA0D481D
:107B600090F86D200DA10F48FCF7DCF901201023DF
:107B70000C4A302100905820FAF756FB07B000BDA0
:107B80003A3B08093A3B56573A3B582459071B5A87
:107B900000010100A41500202300002025303364DB
:107BA000252500009011002000B587B01DA30FCB44
:107BB000CDE90523CDE903011EA00068029002A9CA
:107BC00003A8FDF719FC1C4890F85F0040B10120A4
:107BD00010232A22194600905820FAF74FFA07E09E
:107BE000012010232B22194600905820FAF746FA5C
:107BF000012010236D22194600906820FAF73EFA02
:107C00000D4890F86D200DA10E48FCF78BF901206E
:107C100010230C4A302100905820FAF705FB07B0DA
:107C200000BD00003A3B08093A3B56573A3B5824FE
:107C300059071B5A01000100A415002025303364A8
:107C4000252500009011002000B58BB00EA0006823
:107C50000A900EA0006809900DA0006808900DA081
:107C6000006807900CA207CA04AB07C3062004A94A
:107C700007AA08ABCDE90021029009AA0AA90420AD
:107C8000FEF736FC0BB000BD00010100342E0000F1
:107C9000352E0000362E00003A3B08093C3D3E3FA1
:107CA0004041666710B50246012000E050430B1EBC
:107CB000A1F10104E1B2F9D110BD000000201CE0E7
:107CC0000022254901EB40010A8040F2FF7222495F
:107CD000103101EB40010A8040F6FF721E4920314D
:107CE00001EB40010A8000221B49303101EB800189
:107CF0000A60194950310A54401C0828E0DB022070
:107D00001549891E81F85A001448C1F85B0001200A
:107D100081F85F004FF47A70A1F86000002081F8CC
:107D20006200012081F8630081F8640081F8650039
:107D30000B48C1F86600002081F86A00052081F830
:107D40006B00002081F86C0081F86D0081F86E00F6
:107D50000F2081F86F007047A6150020CDCC6C4035
:107D6000CDCC3C4130B587B004460D4601200F23F1
:107D70001F22002100900846FAF72DF888A000681D
:107D800006900020042306AA014600902020FAF75E
:107D9000E7F901200F237F22002100906020FAF7ED
:107DA0001AF8287810237FA2194600900020FAF7CD
:107DB0003BFA7EA0006805902878022305AA1021CE
:107DC00000902820FAF7CCF9794890F86E00012845
:107DD00016D134B97748007808B9012002E00020B4
:107DE00000E001200E211023734ACDE9001011217B
:107DF0005820F9F7ABFF01217048FBF7F0FD15E0C3
:107E000034B96C48007808B9012002E0002000E095
:107E100001200E2110236A4ACDE9001011215820BB
:107E2000F9F794FF00216548FBF7D9FD6878102326
:107E300064A2202100900020FAF7F6F962A0006801
:107E400004906878042304AA202100901020FAF7F7
:107E500087F9574890F86300012818D1012C06D102
:107E60005448007808B9012002E0002000E0012019
:107E70000E211023504ACDE9001021215820F9F796
:107E800065FF4B4991F86F00F9F70EFE14E0012CE5
:107E900006D14848007808B9012002E0002000E03F
:107EA00001200E211023464ACDE90010212158203F
:107EB000F9F74CFFF9F7B8FDA878102343A2302159
:107EC00000900020FAF7B0F941A000680390A8786C
:107ED000042303AA302100901020FAF741F9344816
:107EE00090F86F000B283BD00D281DD00F2853D1E0
:107EF000022C06D12F48007808B9012002E00020AA
:107F000000E0012010237022302100905820FAF761
:107F1000B5F8274890F86300012804D1244991F866
:107F20006F00F9F7C1FD38E0022C06D12148007836
:107F300008B9012002E0002000E0012010236022A7
:107F4000302100905820FAF799F8194890F863000A
:107F5000012804D1164991F86F00F9F7A5FD1CE03E
:107F6000022C06D11348007808B9012002E0002055
:107F700000E0012010237122302100905820FAF7F0
:107F80007DF80B4890F86300012804D1084991F866
:107F90006F00F9F789FD00E000BF00BF07B030BDFA
:107FA00020210809312E50504D00000020210000F2
:107FB000A4150020230000206600002000080040D7
:107FC00082000020322E000023242526332E0000BC
:107FD0002526272830B589B0002400BF25E044B904
:107FE000002001AA02F8140000216000401C115476
:107FF00019E0082C0FDC601E104931F81000000A4F
:1080000001AA02F81400601E31F81000C1B260002D
:10801000401C115407E0FF2001AA02F81400FF21C0
:108020006000401C1154601C84B2102CD7DB01A8E6
:10803000F9F76EFD0546284609B030BDBC0C00209E
:108040001CB5FCF703FC4FF4A060F9F70DFE4FF4EC
:10805000E13000F0F9FD472140F2CF70FBF7E8F97D
:10806000472144F61F60FBF759FCF8F7CBFFF8F700
:108070005BFDFAF7A7FFFAF7A9FDF8F733FEF9F76A
:1080800013FCF9F763FCFAF715FB1420FCF7CCFBA3
:10809000F9F7BCFEF9F7F2FD2F4890F86500402192
:1080A00080232E4ACDE9001000210846F9F74EFE44
:1080B000F9F73AFF0AE06420FCF7EAFB2848006879
:1080C00008B9012000E0002025490860F9F716FCF6
:1080D0000028F0D1224908604FF47A70FCF7D8FBF1
:1080E000F9F7ECFD1C4890F86C00012822D11D48DE
:1080F0008088B0F5966F15DD1BA000680190012007
:10810000042301AA182100901E20FAF729F8012063
:10811000102316A2182100905E20FAF785F8F9F7CF
:1081200003FF00BF00BF0F488088B0F5966FFADCF0
:10813000F9F7C4FD084890F86300012805D1064905
:1081400091F86F00F9F7B0FC01E0F9F76DFCFCF76E
:10815000FFFCF9F7E9FE1CBDA4150020D2060020A3
:10816000A8012142BC0C00203A3B38392100000014
:108170001CB5002400BF3DE0201D204931F810004F
:1081800040F2E24188420EDA01201221CDE90010CE
:1081900004EB440189000E31C8B20B23184A1221A6
:1081A000F9F7D4FD24E0201D144931F8100040F205
:1081B000D66188420EDA01201221CDE9001004EBCD
:1081C000440189000E31C8B20B230E4A1221F9F77F
:1081D000BDFD0DE001201221CDE9001004EB4401AA
:1081E00089000E31C8B20B23074A1221F9F7AEFD00
:1081F000601CC4B2042CBFDB1CBD0000BC0C002002
:10820000CE010020E6010020FE0100207CB50446DE
:108210000D4620781023FEA2002100900120FAF7DD
:1082200003F8012D17D1FB48D0F83260FA480078E6
:1082300008B9012000E000201021CDE90010002E37
:1082400001DB304600E070420246032300211E207D
:10825000F9F7A0FF11E0EF48D0F8326001201021BB
:10826000CDE90010002E01DB304600E070420246EE
:10827000032300211E20F9F78DFFE648D0F83200D5
:10828000002808DA01201023E4A200210090362003
:10829000F9F7CAFF07E001201023E1A200210090B6
:1082A0003620F9F7C1FF60781023DEA2194600904E
:1082B0000120F9F7B9FF022D17D1D648D0F8366062
:1082C000D548007808B9012000E000201021CDE950
:1082D0000010002E01DB304600E07042024603230E
:1082E00010211E20F9F756FF11E0CA48D0F8366079
:1082F00001201021CDE90010002E01DB304600E006
:1083000070420246032310211E20F9F743FFC148A3
:10831000D0F83600002808DA01201023BFA2194641
:1083200000903620F9F780FF07E001201023BCA25F
:10833000194600903620F9F777FFA0781023BAA2EB
:10834000202100900120F9F76FFF032D17D1B148CC
:10835000D0F83A60B048007808B9012000E0002069
:108360001021CDE90010002E01DB304600E0704204
:108370000246032320211E20F9F70CFF11E0A54837
:10838000D0F83A6001201021CDE90010002E01DB69
:10839000304600E070420246032320211E20F9F7F8
:1083A000F9FE9C48D0F83A00002808DA0120102392
:1083B0009AA2202100903620F9F736FF07E001202D
:1083C000102397A2202100903620F9F72DFFE078A6
:1083D000102396A2302100900120F9F725FF042DEB
:1083E00017D18C48D0F83E608B48007808B901203E
:1083F00000E000201021CDE90010002E01DB304606
:1084000000E070420246032330211E20F9F7C2FE2D
:1084100011E08048D0F83E6001201021CDE9001025
:10842000002E01DB304600E070420246032330217B
:108430001E20F9F7AFFE7748D0F83E00002808DA92
:108440000120102375A2302100903620F9F7ECFEB0
:1084500007E00120102372A2302100903620F9F7A6
:10846000E3FE2079102372A2002100904220F9F748
:10847000DBFE052D17D16748D0F8426066480078CA
:1084800008B9012000E000201021CDE90010002EE5
:1084900001DB304600E070420246032300215F20EA
:1084A000F9F778FE11E05B48D0F842600120102116
:1084B000CDE90010002E01DB304600E0704202469C
:1084C000032300215F20F9F765FE5248D0F84200EF
:1084D000002808DA0120102350A200210090772004
:1084E000F9F7A2FE07E0012010234DA20021009021
:1084F0007720F9F799FE607910234EA21946009073
:108500004220F9F791FE062D17D14248D0F8466077
:108510004148007808B9012000E000201021CDE991
:108520000010002E01DB304600E0704202460323BB
:1085300010215F20F9F72EFE11E03648D0F8466092
:1085400001201021CDE90010002E01DB304600E0B3
:1085500070420246032310215F20F9F71BFE2D48CD
:10856000D0F84600002808DA012010232BA2194673
:1085700000907720F9F758FE07E00120102328A289
:10858000194600907720F9F74FFEA07910232AA210
:10859000202100904220F9F747FE072D17D11D48F2
:1085A000D0F84A601C48007808B9012000E000209B
:1085B0001021CDE90010002E01DB304600E07042B2
:1085C0000246032320215F20F9F7E4FD11E0114862
:1085D000D0F84A6001201021CDE90010002E01DB07
:1085E000304600E070420246032320215F20F9F765
:1085F000D1FD0848D0F84A0000281FDA01201023D6
:1086000006A2202100907720F9F70EFE1FE000005F
:1086100043483100A4150020230000202D00000055
:108620002B000000434832004348330043483400E5
:1086300043483500434836004348370001201023A3
:10864000AFF22402202100907720F9F7EDFDE079C8
:10865000102325A2302100904220F9F7E5FD082DD6
:1086600017D12248D0F84E602148007808B901207F
:1086700000E000201021CDE90010002E01DB304683
:1086800000E070420246032330215F20F9F782FDAB
:1086900011E01648D0F84E6001201021CDE90010FD
:1086A000002E01DB304600E07042024603233021F9
:1086B0005F20F9F76FFD0D48D0F84E00002809DA69
:1086C00001201023AFF2AC02302100907720F9F79F
:1086D000ABFD08E001201023AFF2BC023021009076
:1086E0007720F9F7A1FD7CBD43483800A415002090
:1086F0002300002038B504460D462078102363A2DD
:10870000002100900120F9F78FFD012D06D160486E
:10871000007808B9012002E0002000E001201023C9
:108720005CA2002100902820F9F77EFD60781023DC
:1087300059A2194600900120F9F776FD022D06D1C5
:108740005348007808B9012002E0002000E0012031
:10875000102352A2194600902820F9F765FDA07851
:1087600010234FA2202100900120F9F75DFD032D79
:1087700006D14748007808B9012002E0002000E057
:108780000120102347A2202100902820F9F74CFD5A
:10879000E078102344A2302100900120F9F744FD35
:1087A000042D06D13A48007808B9012002E00020E3
:1087B00000E0012010233DA2302100902820F9F78D
:1087C00033FD207910233AA2002100904220F9F7CE
:1087D0002BFD052D06D12E48007808B9012002E0B6
:1087E000002000E00120102332A200210090692027
:1087F000F9F71AFD607910232FA219460090422044
:10880000F9F712FD062D06D12148007808B901209C
:1088100002E0002000E00120102328A21946009069
:108820006920F9F701FDA079102325A220210090ED
:108830004220F9F7F9FC072D06D11548007808B950
:10884000012002E0002000E0012010231DA22021D1
:1088500000906920F9F7E8FCE07910231AA2302192
:1088600000904220F9F7E0FC082D06D10848007876
:1088700008B9012002E0002000E00120102313A22B
:10888000302100906920F9F7CFFC38BD4348310012
:1088900023000020593100004348320059320000C3
:1088A0004348330059330000434834005934000032
:1088B000434835004B310000434836004B3200003E
:1088C000434837004B330000434838004B34000026
:1088D0007CB505460C4628781023CFA200210090D5
:1088E0000120F9F7A1FCCD4890F85200012813D1DE
:1088F000012C06D1CA48007808B9012002E0002006
:1089000000E001200E211023C64ACDE9001001210C
:108910001E20F9F71BFA12E0012C06D1C04800789E
:1089200008B9012002E0002000E001200E21102300
:10893000BD4ACDE9001001211E20F9F707FA687839
:108940001023BAA2194600900120F9F76DFCB34834
:1089500090F85300012813D1022C06D1B0480078BA
:1089600008B9012002E0002000E001200E211023C0
:10897000AC4ACDE9001011211E20F9F7E7F912E009
:10898000022C06D1A648007808B9012002E0002098
:1089900000E001200E211023A34ACDE9001011218F
:1089A0001E20F9F7D3F9A8781023A1A22021009066
:1089B0000120F9F739FC994890F85400012813D1A7
:1089C000032C06D19648007808B9012002E0002067
:1089D00000E001200E211023924ACDE90010212150
:1089E0001E20F9F7B3F912E0032C06D18C48007869
:1089F00008B9012002E0002000E001200E21102330
:108A0000894ACDE9001021211E20F9F79FF9E87865
:108A1000102388A2302100900120F9F705FC7F483F
:108A200090F85500012813D1042C06D17C48007819
:108A300008B9012002E0002000E001200E211023EF
:108A4000784ACDE9001031211E20F9F77FF912E0B4
:108A5000042C06D17248007808B9012002E00020F9
:108A600000E001200E2110236F4ACDE900103121D2
:108A70001E20F9F76BF9287910236FA200210090CE
:108A80004220F9F7D1FB654890F85600012813D130
:108A9000052C06D16248007808B9012002E00020C8
:108AA00000E001200E2110235E4ACDE900100121D3
:108AB0005E20F9F74BF912E0052C06D158480078F2
:108AC00008B9012002E0002000E001200E2110235F
:108AD000554ACDE9001001215E20F9F737F9687990
:108AE000102356A2194600904220F9F79DFB4B48EF
:108AF00090F85700012813D1062C06D14848007879
:108B000008B9012002E0002000E001200E2110231E
:108B1000444ACDE9001011215E20F9F717F912E05F
:108B2000062C06D13E48007808B9012002E000205A
:108B300000E001200E2110233B4ACDE90010112155
:108B40005E20F9F703F9A87910233DA220210090B7
:108B50004220F9F769FB314890F85800012813D1F9
:108B6000072C06D12E48007808B9012002E0002029
:108B700000E001200E2110232A4ACDE90010212116
:108B80005E20F9F7E3F812E0072C06D124480078BC
:108B900008B9012002E0002000E001200E2110238E
:108BA000214ACDE9001021215E20F9F7CFF8E879BC
:108BB000102324A2302100904220F9F735FB1748FA
:108BC00090F85900012813D1082C06D114480078D8
:108BD00008B9012002E0002000E001200E2110234E
:108BE000104ACDE9001031215E20F9F7AFF812E00C
:108BF000082C06D10A48007808B9012002E00020BC
:108C000000E001200E211023074ACDE90010312198
:108C10005E20F9F79BF87CBD43483100A415002085
:108C2000230000206600002082000020434832001C
:108C30004348330043483400434835004348360036
:108C4000434837004348380010B586B00446012138
:108C500044F20900F9F7A6FD01210420F8F7EAFC27
:108C60002248FAF7E5FF4020ADF8140003208DF804
:108C7000160018208DF8170005A91D48F8F74EFCBE
:108C80008020ADF8140004208DF8170005A91848BD
:108C9000F8F744FC01940020ADF80800ADF80A0094
:108CA000ADF80C00ADF810000C20ADF80E0001A9D5
:108CB0000E48FBF75BF825208DF8000003208DF8A7
:108CC00001008DF8020001208DF803006846F8F7D6
:108CD00093FF012240F225510448FBF721F80121BE
:108CE0000248FAF799FF06B010BD000000380140B5
:108CF000000C014048000000000C01402000000072
:108D00000800000048000000000C014010000000B6
:108D10000800000048000000000C014008000000AE
:108D2000080000004800000000080140008000002A
:108D3000040000004800000000080140001000008E
:108D40000400000048000000000801400008000086
:108D50000400000048000000000C01400008000072
:108D600008000000344310100134431010010000CB
:108D700000000000000000000000000000003F4074
:108D80000000000000000000300040003000400003
:108D9000000009000BC03D000BC03D00090018C0D9
:108DA00024407FE0224031800000180024C01B00D6
:108DB0000D803240018003801C4027401C8007400A
:108DC00000401000600000000000000000000000F3
:108DD000000000001F802040402000004020204074
:108DE0001F8000000000090006001F800600090027
:108DF0000000040004003F80040004000000001094
:108E000000600000000000000000040004000400F6
:108E1000040004000000000000400000000000000A
:108E20000000002001C006003800400000001F8044
:108E30002040204020401F800000000010403FC024
:108E400000400000000018C021402240244018408B
:108E5000000010802040244024401B8000000200BD
:108E60000D0011003FC0014000003C802440244020
:108E70002440238000001F8024402440344003808D
:108E800000003000200027C03800200000001B80B8
:108E90002440244024401B8000001C0022C02240AB
:108EA00022401F8000000000000008400000000079
:108EB000000000000000046000000000000000004E
:108EC00004000A0011002080404009000900090048
:108ED00009000900000000004040208011000A0045
:108EE00004001800200023402400180000001F8008
:108EF0002040274029401F400000004007C03900A3
:108F00000F0001C0004020403FC0244024401B808F
:108F100000001F8020402040204030800000204082
:108F20003FC0204020401F80000020403FC0244020
:108F30002E4030C0000020403FC024402E003000B2
:108F400000000F00108020402240338002002040AB
:108F50003FC0040004003FC02040204020403FC0EC
:108F60002040204000000060202020203FC0200042
:108F7000200020403FC024400B0030C02040204053
:108F80003FC020400040004000C03FC03C0003C044
:108F90003C003FC0000020403FC00C4023003FC0C9
:108FA00020001F802040204020401F8000002040E3
:108FB0003FC024402400180000001F8021402140B1
:108FC00020E01FA0000020403FC02440260019C020
:108FD000004018C02440244022403180000030006E
:108FE00020403FC020403000000020003F80004073
:108FF00000403F80200020003E0001C007003800F4
:109000002000380007C03C0007C0380000002040A6
:1090100039C0060039C0204000002000384007C099
:10902000384020000000304021C02640384020C099
:109030000000000000007FE0402040200000000011
:1090400070000C0003800040000000004020402021
:109050007FE0000000000000200040002000000031
:1090600000000010001000100010001000100000A0
:1090700000004000000000000000000002800540E9
:10908000054003C0004020003FC00440044003806E
:10909000000000000380044004400640000000007F
:1090A0000380044024403FC000400000038005408E
:1090B000054003400000000004401FC0244024403D
:1090C0002000000002E0055005500650042020401A
:1090D0003FC00440040003C000400000044027C01B
:1090E00000400000000000100010041027E0000005
:1090F000000020403FC00140070004C00440204061
:1091000020403FC000400040000007C0040007C0EE
:10911000040003C00000044007C00440040003C072
:10912000004000000380044004400380000004105D
:1091300007F0045004400380000000000380044056
:10914000045007F00010044007C00240040004006F
:109150000000000006400540054004C0000000007B
:1091600004001F800440004000000400078000400D
:10917000044007C000400400070004C0018006004E
:109180000400060001C0070001C006000000044002
:1091900006C0010006C0044000000410071004E0EF
:1091A0000180060004000000044005C006400440A1
:1091B00000000000000004007BE0402000000000F0
:1091C00000000000FFF000000000000040207BE0F5
:1091D000040000000000400080004000200020004B
:1091E000400000000000000000000000000000003F
:1091F00000000000000000001FCC000C0000000078
:10920000000000000800300060000800300060002E
:109210000000022003FC1E20022003FC1E2002206E
:10922000000000000E1811043FFF10840C780000AD
:1092300000000F0010840F3800C0077818840078F1
:10924000000000780F8410C411240E9800E40084FC
:109250000008080068007000000000000000000026
:10926000000000000000000007E018182004400281
:109270000000000040022004181807E00000000071
:1092800000000240024001800FF0018002400240D5
:1092900000000080008000800FF8008000800080C7
:1092A00000000001000D000E0000000000000000A2
:1092B00000000000008000800080008000800080AE
:1092C00000800000000C000C000000000000000006
:1092D0000000000000060018006001800600180071
:1092E0002000000007F0080810041004080807F028
:1092F00000000000080408041FFC00040004000033
:10930000000000000E0C10141024104411840E0CE8
:10931000000000000C1810041104110412880C70D5
:109320000000000000E00320042408241FFC0024A7
:10933000000000001F9810841104110410881070A0
:109340000000000007F0088811041104188800705C
:10935000000000001C00100010FC13001C00100096
:10936000000000000E3811441084108411440E389F
:10937000000000000700088C10441044088807F023
:109380000000000000000000030C030C00000000BF
:1093900000000000000000010106000000000000C5
:1093A00000000000008001400220041008081004A2
:1093B00000000220022002200220022002200220BF
:1093C0000000000010040808041002200140008082
:1093D000000000000E001200100C106C10800F0036
:1093E000000003E00C1813E4142417C4082807D065
:1093F00000000004003C03C41C40074000E4001CC3
:10940000000410041FFC1104110411040E880070E4
:10941000000003E00C1810041004100410081C10C5
:10942000000010041FFC100410041004080807F0CA
:10943000000010041FFC1104110417C410040818C4
:10944000000010041FFC1104110017C010000800D8
:10945000000003E00C181004100410441C780040B5
:10946000000010041FFC10840080008010841FFC8A
:1094700010040000100410041FFC1004100400006D
:10948000000000030001100110011FFE1000100079
:10949000000010041FFC110403801464181C100445
:1094A000000010041FFC1004000400040004000C61
:1094B000000010041FFC1F0000FC1F001FFC100414
:1094C000000010041FFC0C04030000E010181FFC37
:1094D000100007F00808100410041004080807F032
:1094E000000010041FFC10841080108010800F00FA
:1094F000000007F0081810241024101C080A07F2B6
:10950000000010041FFC1104110011C011300E0CDA
:10951000000400000E1C11041084108410441C3838
:1095200000001800100010041FFC100410001800A8
:10953000000010001FF810040004000410041FF8BD
:10954000100010001E0011E0001C007013801C00B1
:1095500010001FC0103C00E01F0000E0103C1FC0C6
:1095600000001004180C163401C001C01634180C89
:10957000100410001C00130400FC13041C00100055
:1095800000000804101C1064108413041C0410183C
:1095900000000000000000007FFE40024002400288
:1095A0000000000030000C0003800060001C00037D
:1095B000000000004002400240027FFE0000000068
:1095C000000000000000200040004000400020009B
:1095D0000000000100010001000100010001000184
:1095E00000010000400040002000000000000000DA
:1095F000000000000098012401440144014400FCE3
:10960000000410001FFC00880104010400880070A1
:1096100000000000007000880104010401040088BB
:1096200000000000007000880104010411081FFC04
:109630000004000000F8014401440144014400C852
:1096400000000000010401040FFC110411041100CA
:109650001800000000D601290129012901C90106CD
:10966000000010041FFC008401000100010400FC44
:10967000000400000104190419FC000400040000A7
:1096800000000000000300010101190119FE0000A3
:10969000000010041FFC0024004001B4010C010470
:1096A00000000000100410041FFC0004000400006F
:1096B0000000010401FC0104010001FC010401009F
:1096C00000FC010401FC008401000100010400FC15
:1096D0000004000000F8010401040104010400F882
:1096E0000000010101FF00850104010400880070F1
:1096F000000000000070008801040104010501FF62
:1097000000010104010401FC008401040100018046
:109710000000000000CC0124012401240124019850
:10972000000000000100010007F80104010400002E
:109730000000010001F8000400040004010801FC1D
:109740000004010001800170000C00100160018024
:10975000010001F0010C003001C00030010C01F0EB
:10976000010000000104018C00740170018C0104EF
:109770000000010101810171000E001801600180EB
:10978000010000000184010C013401440184010C3A
:109790000000000000000000000001003EFC40024C
:1097A00040020000000000000000FFFF0000000079
:1097B00000000000400240023EFC010000000000EA
:1097C0000000000060008000800040004000200099
:1097D0002000000000000000000000000000000069
:1097E0000000000000000000000000000000000079
:1097F0000000000000000000000000000000000069
:109800000000000000000000000000000000000058
:109810000000000000000000000000000000000048
:10A520000000000000000000000000000000881093
:10A530004FE000109FD09510D510BFD0B510D5506A
:10A540001FD0001000000201420233FC0002000193
:10A5500047FF4491549154914FFD54916495449315
:10A5600007FD0001000002000202420433F800046B
:10A57000100297FA55521D5215521552555297FA1C
:10A580001002000200000880110023FFCC0101022C
:10A59000797C0940F940097C790804111BE6E81828
:10A5A0000FE6080100000200420033FC0008001121
:10A5B0007FFE4100497849487F484948497A41012E
:10A5C0007FFE0000000000024002400243FE400205
:10A5D000400240027FFE410241024102410241022B
:10A5E0004002000200000002000C3FF1240124029E
:10A5F000270224C42428441044284444C582460227
:10A6000000010001000008200620407E318000008B
:10A610007F7F4911491249124900497E4909491170
:10A620007F1100270000084008420881FFFE090052
:10A6300004021902124214429042707E14421242E5
:10A6400015421802000002000200420033FC00091B
:10A650000211050279C24134410841147962058230
:10A660000401040100000002E802A802ABFEAAAA4D
:10A67000EAAAAAAABEAAAAAAEAAAAAAAABFEA802FB
:10A68000E802000200000004200421042104210447
:10A690002104210421042104210421042104210492
:10A6A0002004000400000401080617F82490E49038
:10A6B0002490249027FE24902C903492049107FE3D
:10A6C00000000000000000049004D7D4A555A55652
:10A6D000857CFD5407D49554D57CA556A55587D4C3
:10A6E000F804000400000082208424882491A4A19E
:10A6F00064D127913C91249F6491A4912491249149
:10A7000020810080000002000202420433F80004AD
:10A7100020122F2229422982FFFA298229422F2240
:10A720002012000200001080110097FF58800342A1
:10A73000242428A8FEA228A104BE28A0FEA028A8A0
:10A74000242402020000000040FF5E9252925292C6
:10A7500052FE529252925E9240FF00000FF00002B1
:10A760000001FFFE0000082008220841FFFE0880CB
:10A770000A4122412A52A66A63C42244264A2A7206
:10A7800022410240000000003FF000200040FFFF97
:10A790000000020104021B84E868081008680F84A6
:10A7A00008020801000011002600C40045FF6552A0
:10A7B000555245525D522552C55245D2641F540030
:10A7C0004500460000002004210621043FF821082E
:10A7D000210800027F22492249227FFE4922492284
:10A7E0007F2200020000020422482A52A64163FE92
:10A7F00026402A50224900063FF82200220023FF6B
:10A800004200020000002001212223142D1831E40F
:10A8100008142A922A922A92FFFE2A922A923E92A3
:10A8200008120802000002000202420433F8000489
:10A830000A0A723213C21202FE0213F2120A120A3A
:10A84000023A0002000008420841FFFE08800000B2
:10A850004108614852484A4845FF4A4852486148C1
:10A86000010801000000082008C00B00FFFF0900DC
:10A87000289127D2F554255825702558F55427D20C
:10A880002011000100000422444245927E1244122D
:10A8900044127F92447E441200123E1200920052F3
:10A8A000FF82000200000080010006001FFFE0049C
:10A8B00000887C9044A044C047FF44C044A07C90E2
:10A8C00000880004000020402080210027FF38007D
:10A8D000E04024402442244124FE254026402440D8
:10A8E0002040204000000080010006001FFFE00023
:10A8F00000002000249F2492A49264922492249227
:10A90000249F2000000008403140225E20822782E0
:10A9100020C2A942657E22422442284221C2221F2F
:10A920002900300000002040218027FE3A0822083C
:10A9300023FC000040104F104110411041127F11C4
:10A94000010201FC000011901698F89013FF10A06E
:10A95000080013FF2A484A498BFF480029FA1001D2
:10A960000BFE080000000000003E3E020202020250
:10A9700002020202FFFE02020202020202023F0281
:10A98000003F000000000001000200040008003049
:10A9900080C047003800070000C00030000C0002F3
:10A9A000000100010000000102024204420842309E
:10A9B00043C07E00420043FC4202420242020202C5
:10A9C000020E0000000004440CE63544C64804486A
:10A9D0001848010209020904FFC8093092285244AC
:10A9E0001282021F0000000000041808683108C12C
:10A9F0000B011D82E962091409080914492229C2C0
:10AA0000080100010000004000423FC46A48AA5209
:10AA10002A613FFE00000800088008620801FFFE6E
:10AA20000800080000001008100C10081FF8101093
:10AA300010111012080C0870FF80080208010802AB
:10AA40000FFC000000000010289025102210249018
:10AA50002C90B59066BF2490299020D0221025100C
:10AA600028900010000000003FF8221022103FF84C
:10AA7000000000411FC210441058FFE0105810445D
:10AA80001FC2004100001004100810121062118251
:10AA90001E82F082108210FE1082108210821082BC
:10AAA000100210020000101010201040108013FF40
:10AAB0001C82F0821082108210821082108210FF9D
:10AAC00010001000000002000201420233FC0002EC
:10AAD000000152814CBD448554858FFD84858C8551
:10AAE000B4BD00810000082008C00B00FFFF090072
:10AAF00008C001004100410041007FFF41004100CA
:10AB0000410001000000010041014102410C7FF0C1
:10AB1000410041004100410041007FFF41004100F0
:10AB20004100010000000081008108828882688461
:10AB3000088808B00FC008B008882884C882088236
:10AB4000008100810000010101063FF86940A73241
:10AB500021013FFE00001C0013FC90227042108275
:10AB60001502181E00000400040104017DF555556E
:10AB70005555555555FF5555555555557DF50401B8
:10AB8000040104000000000200027E7E0042004238
:10AB9000FF7E004202420C42F07E20422842267E86
:10ABA00020020002000010401080910077FF190081
:10ABB00000C100027FC4401840604F80407E4001C9
:10ABC0007FC1000700000000004244444CC854D03C
:10ABD00065424541467E844088409050814880C40B
:10ABE00000620000000004440CE63544C6480C48EE
:10ABF00000011102130C15F09900710011FC1502EF
:10AC00001302118E000004001800107C57403540DC
:10AC100015401540F5FF154015403548574410784C
:10AC2000140018000000000100067FF84440444072
:10AC3000444044407FFE44404440444244417FFEFF
:10AC4000000000000000082008220841FFFE0880E4
:10AC5000090000007FFF410141C2413449084534E9
:10AC600079C20001000048405740F55755555755E7
:10AC7000F0D55F5540D511553155EA5524552A5721
:10AC800031402140000008200620407E3180000035
:10AC90000FFF084208420842FFFE084208420842ED
:10ACA0000FFF0000000000001FFF80006000000098
:10ACB00000004000400040004000400040024001D1
:10ACC0007FFE0000000000400880110023FFCC0040
:10ACD0000000020042004202420143FE42004200E4
:10ACE0004200020000002410246025807FFFC48001
:10ACF000446000027C924492449244FE4492449206
:10AD00007C9200820000082008C00B00FFFF0900B1
:10AD100008800101120114C290347008103414C26A
:10AD20001201110100000020402030FE0700020047
:10AD300004001FFFF244124492447FFC1244124468
:10AD4000124410040000008007000000FFFF08000C
:10AD50000408103011C11E22F0C4101817E010189A
:10AD6000104611810000040108091009EF922AB26F
:10AD70002AEA2AA42AA42AA42AAA2AB22FA22001B3
:10AD8000200100010000000100067FF840004000A3
:10AD900040004000400040004000400040004000B3
:10ADA0004000400000000200020042004200420059
:10ADB000420242017FFE4200420042004200420045
:10ADC000020002000000000800081FC89248524814
:10ADD000324812481FFF12483248524892481FC852
:10ADE0000008000800000080010006001FFFE002CC
:10ADF00008020982087A88026802080E08720B822B
:10AE0000080200020000084008420881FFFE090015
:10AE100004001901112111D297147108111411E2C3
:10AE200015011900000002800C80F7FE2484248A9A
:10AE30000164271839E408222AA22AA2FFFA2AA2CA
:10AE40003EA20822000002000200220022FF2A92F5
:10AE50002692A2926292229226922A9222FF2200A7
:10AE600002000200000011021204148890505020C9
:10AE700014D0120C110101020E04F1C8103010CCD4
:10AE80001F0210010000082008C00B00FFFF09008E
:10AE900008C100067FF84000400040007FFC00022F
:10AEA0000002001E000040004FFE400240024FF230
:10AEB000491249124FF2491249124FF24002400220
:10AEC0004FFF400000004000400047FF44024402A2
:10AED0004FFE74924492449247FE4402440247FF5C
:10AEE000400040000000000000F83C9024902490B6
:10AEF00024902490FFFF24902490249024903C9050
:10AF000000F800000000000000003FFE20042004C4
:10AF100020042004200420042004200420043FFEF8
:10AF200000000000000002000200420033FC0008A4
:10AF30000914090609FC09080908FF800870880C33
:10AF40006802080F0000000000001FF81110111027
:10AF500011101110FFFE11111111111111111FF912
:10AF60000001000F0000000100067FF840024102CE
:10AF70004102410241025FFE410241024122411A67
:10AF800041024002000000001FFF8000440004F85E
:10AF9000448054804FFE4490448844F04402400171
:10AFA0007FFE00000000048008803480E7FE2484D7
:10AFB000248800000FE008400840FFFF08400840D8
:10AFC0000FE00000000000003FFC210821082108DC
:10AFD0003FFC000008000880086008020801FFFE2E
:10AFE0000800080000000100010001000100FFFF4F
:10AFF00001020184054809201110210841040104BF
:10B00000010201020000010006001FFFE002003CF7
:10B010003FC024FF2490A4FE649024FE2490249139
:10B020003CFF00000000080208440FA8F810086860
:10B030000F86000001004102410147FE4900510016
:10B0400061000100000000000FFF084208420842B2
:10B05000FFFE084208420842FFFE0842084208423A
:10B060000FFF00000000008102810C8278840888B4
:10B0700008B008C0FF8008C008B0088808840882AB
:10B08000008100810000082008220841FFFE08819D
:10B090000902000C1FF01100910071001100110055
:10B0A00011001F8000000000000000001FFF11229F
:10B0B0003122512291221122112211221FFF000060
:10B0C000000000000000082008C00B00FFFF09007E
:10B0D0000A8204220A1A3282C27232060A1A04E270
:10B0E0000202020200000200420033FE00040008D7
:10B0F00022002AFF2AA82AA8FEA82AAA2AA92AFEEC
:10B10000220002000000002010200C400080FFFF01
:10B11000000011402150CA484442484153FE60405B
:10B12000004000400000000000007FFE400440049A
:10B130004FE44824482448244FE4400440047FFE60
:10B14000000000000000000000000FF008200820B0
:10B1500008200820FFFF08200820082008200FF002
:10B1600000000000000002000400080037FCE44278
:10B1700024422442244227C2202220123FE200021D
:10B18000000E00000000082008220841FFFE088091
:10B1900009000400247F244224427FC24442C44266
:10B1A000447F0400000000003FFC04442484150494
:10B1B000FFF4150424C500063FF82200220023FFF7
:10B1C00042000200000004440CE63544C64808482A
:10B1D00000007FFE12220A420282FFFE02820A4221
:10B1E00012220002000004440CE63544C64804481C
:10B1F00018480411245125322494FC1825F02418F1
:10B200002514061300007E9752904A967FE04AA6C6
:10B2100052A07EAD0402040C0470FF800470440C44
:10B2200034020401000002000200420033FC000965
:10B2300000120004001800E0FF0000E00018000405
:10B2400000020001000000007FFF4002441244227F
:10B250004442448A45065FFA4402440244024002E2
:10B260007FFF0000000000007FFF401044085B11DA
:10B2700060E20004001800E0FF0000E00018000495
:10B280000002000100002002202222242324F2A830
:10B2900022302220237F24202430F4A82D242424AB
:10B2A0002022200200000008081008200840089012
:10B2B0000B100C10FFFF0C100B100890084008201A
:10B2C000081000080000000100061FF81100110816
:10B2D000110411F810011002FF84106890185064D6
:10B2E0001382101F00000000004002401240124074
:10B2F0001240324232423FFE22402240224022404F
:10B300002240004000000010101011901290149084
:10B310001890F09017FF10901090109010901090CF
:10B32000101000100000010101063FF86940A7322B
:10B3300021013FFE0100027F7C42404240427E42AA
:10B34000027F020000002000207F204020402F5E6E
:10B350002952A9526952295229522F5E2040204178
:10B36000207F200000000080010006001FFFE00099
:10B3700000003FFF2102210421007F824171C10CA6
:10B380004102011F000000000000200400200C10FA
:10B3900020180E2010063FE00000100000080000FA
:10B3A0000C21FFF42122042122062922062522064F
:10B3B00027FFF62722062922062922063122161106
:10B3C000223E01FFF6000004000000000000000320
:10B3D000030601040602050003051F1C1F1E1F1E95
:10B3E0001F1F1E1F1E1F000008B4000800000020C1
:10B3F000300B0000180A0008D4BA0008300B0020F7
:10B40000E80E00005C3F00080124B201380D040C76
:10B41000183060C06030180C048007290F1B8001B1
:10B4200024101A028002C004BC056C05E80B900BC6
:10B43000100E081C081C18186033803C1220481D90
:10B440007FF8FFFCC00CC20CC70CC38CC1CCC1CCB4
:10B45000C38CC70CCE0C9C0C39FC13F81C1815C8F7
:10B460004CDCECCFCCC78CC78CCFCCDCECC84CC050
:10B470000CFFFC1A69024AE8024BC008024819FF97
:10B48000F8DFC8DF88DF08DE08DC08D868C0E8C15C
:10B49000E8C3E8C7E8FFF81E4808DE68DEE8DDE834
:10B4A000D92E7A1844100BF8FFF0FFE0FFC0FF80A0
:10B4B000FF12FE12FC12F812F012E012C022801AE3
:10B4C0007002112503F003F01C1FF01F06192A0A51
:10B4D00010F016ADAAA0555016AD0AA01550161CB6
:10B4E00002A0011099161220190AE91616FE70BA68
:10B4F00070D61EEFF0D7F0BA68696E180EEFB0DFA5
:10B50000F0BDE07DF07DF001F07F021CBFE0DF14B4
:10B5100011280AC01FC03FC07FC07FE0241C7FE00D
:10B520007F0E1B1FC0B5101AD01FA03F407E807D2C
:10B5300060FAF0F5F06BE057C02FC05FC080C03FED
:10B54000FF280A7FF980FFF0C0FFE040031BF0C036
:10B550000F1915291828083F80FE1FC0FC0F03197A
:10B5600009190F4918380867FF80C3FFC081031904
:10B5700009190F19151112101A300212383A7802EF
:10B5800012FC480BFF01FC01FC037C037C02022A35
:10B59000FC02680803FC03FE03FE010212FF1AFF0F
:10B5A0002A29022AF8021A01021E03F807F00FE402
:10B5B0001A3FBC1808FFE0FEE0FCC0F0BD4280125C
:10B5C000084AE822380903800738067C0EFE022864
:10B5D000087C0F380F800FF8023A1F02780A17F81C
:10B5E00037F827F867F847023A4F02101A6F806F52
:10B5F000383E7C3EFE3EFE1EFE1E7C3F387F807F36
:10B60000E06FC06F8040524012011D018001C002F6
:10B610001AE0025AF0023994190219CC690219C4CD
:10B6200039023A07025C0FFC1F161A070649141963
:10B63000021CF407FE043AF0E692F0420113514B6B
:10B6400046080102090A130D73460802030112138A
:10B65000857546080304021A136D6C460804050339
:10B660001E13B56D46080506042213ED7146080643
:10B6700007052513497446080708062D1341684637
:10B68000080809072E13757A46080901084413B9FA
:10B690006A2E080A0B110A791A696C2D0B0C0A0B19
:10B6A0000C1A850C2D0C0D0B0C0C1AA10C2D0D0E6B
:10B6B0000C0D0C1ABD0C2D0E0F0D0E0C1AD90C2DE5
:10B6C0000F100E0F0C1AF50C2D10110F100C1A1173
:10B6D000782D110A10110C1A2D0C361213191202A2
:10B6E0001AE1C02D131412130C1AFD0C2D1415138E
:10B6F000140C1319762E08151614150C1A350C2D6A
:10B70000161715160C1A510C2D171816170C1A6D42
:10B710000C2D181917180C1A890C2D191218190C40
:10B720001AA50C2E1A1B1D1A03F012722E081B1CD0
:10B730001A1B0C1AD9182D1C1D1B1C0C13CD672E9F
:10B74000081D1A1C1D0C13C96C37081E1F211E046E
:10B75000135D7A2E081F201E1F0C1AD10C2D2021DC
:10B760001F200C13E1662E08211E20210C1AC1484F
:10B7700036222324220513D5711A080B2A230C1311
:10B78000A1771A080B3A240C126A2F0825262C25BB
:10B79000069019F02D262725260C1AC10C2D2728D6
:10B7A00026270C1ADD0C2D282927280C1AF90C2D18
:10B7B000292A28290C1315752E082A2B292A0C1A38
:10B7C000310C2D2B2C2A2B0C1A4D0C2D2C252B2C0F
:10B7D0000C1A690C362D2D2D0707139D6837082E7E
:10B7E0002F3334081AE5D82D2F302E370C1A458404
:10B7F0002D30312F3A0C1A79A82D3132303D0C13EF
:10B80000497C2E08323331400C1AB9B42D332E3214
:10B81000420C13816B3708343536342E1AF1E41993
:10B820000B2A350C1A25FC190B2A360C13116E370E
:10B8300008373839372F1371691A080B2A380C1A50
:10B84000F924190B2A390C13E16C37083A3B3C3ABE
:10B850003013AD6F1A080B2A3B0C1399701A080BA2
:10B860002A3C0C1AC148363D3E3F3D3113E97A1A55
:10B87000080B2A3E0C13A97B1A080B2A3F0C1361F4
:10B88000722F0840404041326C12792E08414141EC
:10B89000320C131578370842424243331ADDB42D77
:10B8A000434343330C1A49782E444444090924196C
:10B8B0001881120A120B120C120D120E120F121016
:10B8C0001211121212131214121512161217121844
:10B8D0001219121E121F12201221122212231224D8
:10B8E00012251226122712281229122A122B122C84
:10B8F000123412351236123712381239123A123BFC
:10B90000123C123D123E123F0A50FF015ADF085A04
:10B91000CF085AC7084BC3FB084BC1F3085BC0E311
:10B92000085A4308110A2D1F08114A7F085A3F0878
:10B930005A7F084AFF085A01085A03082C07FF07D4
:10B94000084B800F9B19471A9F0712FE3C3FFFBF11
:10B95000083A7F0812FC3AFF183BF801C3180BFBAA
:10B96000F803FFFFE7FFFFF9F03D19BA1CF8E00FFD
:10B970000D19081A60861AFC08112B3FF08912F87D
:10B980003A7FE912F8393E193F3BFE3F081A03257A
:10B9900029084B07F1082D0FE7FFFD081E1F8FFF39
:10B9A000FCE108380B3FBFFFFC6BFFFFF07F9F08F7
:10B9B0001AE07529081AE1751EFC65FFFFC3BF1A5E
:10B9C000FCC02A876F1D61FFFF8E0C29202A18AB4F
:10B9D00019084A33082BFE47082F61FFFC1FFFC0E0
:10B9E0008F2BFC3F081C61FFF8F8211B6DFF7D3990
:10B9F000085AF708190119085A7108195439081911
:10BA000060A90129703EFFFFC7FFF8305CC7FFF057
:10BA1000085AE0085AC0203A80404BC7FF485BC72D
:10BA2000FE084AFC504BC7F8704CC7F004084BE0C6
:10BA30000C084BC01C084B803C30113A7C3012C0C3
:10BA40004AFCA05A01085A03084A07904CC00FFC50
:10BA5000B05A1F103C3FFC6F084C7FFCEFB85AFDFA
:10BA600008DBFFE1E0492889085970F91859C84AEC
:10BA70000CC04CFC1C6BC84A3C084BF07C083CE0FA
:10BA8000FC65084AC1904BC783904BC707B05BC6A3
:10BA90000FB82169086970699069104AFD085A0158
:10BAA000083A030829C95908095801A132384DF448
:10BAB00001E803042902690CA90453401F84A24A27
:10BAC00004680901020304060708090C691005004F
:04BAD000020406085E
:0400000508000101ED
:00000001FF
